:1080000000400020D911010021E7000021E7000015
:1080100021E7000021E7000021E700000000000048
:1080200000000000000000000000000021E7000048
:1080300021E700000000000021E70000FD850000AE
:1080400021E7000021E7000021E7000021E7000010
:1080500021E7000021E7000021E7000021E7000000
:1080600021E7000021E7000021E7000021E70000F0
:1080700021E7000021E7000021E7000021E70000E0
:1080800021E7000021E7000021E7000021E70000D0
:1080900021E7000021E7000021E7000021E70000C0
:1080A00021E7000021E7000021E7000021E70000B0
:1080B00021E7000021E7000021E7000021E70000A0
:1080C00021E7000021E7000021E7000021E7000090
:1080D00021E7000021E7000021E7000021E7000080
:1080E00021E7000021E7000021E7000021E7000070
:1080F00021E700005187000021E7000021E7000090
:1081000021E7000021E7000021E7000021E700004F
:1081100021E7000021E7000021E7000021E700003F
:1081200021E7000021E70000C1DE000021E7000098
:1081300021E7000021E7000021E7000021E700001F
:1081400021E7000021E7000021E7000021E700000F
:1081500021E7000021E7000021E7000021E70000FF
:1081600021E7000031F9000021E7000021E70000CD
:1081700021E7000021E7000021E7000021E70000DF
:1081800021E7000021E7000021E7000021E70000CF
:1081900021E7000021E7000021E7000021E70000BF
:1081A00021E7000021E7000021E7000021E70000AF
:0C81B00021E7000021E7000021E70000AB
:10840000FFFFFFFFFFFFFFFFFFFFFFFF7EF9FFFF03
:1084100010B5054C237833B9044B13B10448AFF3BE
:1084200000800123237010BD00C6FF1F0000000064
:10843000A81601000C4B43B10C480D4910B5AFF321
:1084400000800C48036823B910BD0A48036833B99B
:108450007047094B002BF7D0BDE810401847064B7A
:10846000002BF5D0184700BF00000000A81601003F
:1084700004C6FF1F74C5FF1F0000000080F31188B1
:1084800070472F4B41F238015A5842F478525A50F3
:108490002C4A927902F00C020C2A4FD041F244028D
:1084A0002949995003F558339A78110748BF9A78AB
:1084B000264944BF42F008029A70214B41F244021F
:1084C000995041F204015A5842F4803242F0C002FD
:1084D0005A501A6842F440221A6003F5E833242205
:1084E0005A701B4A80211170A2221A70DA7802F0A9
:1084F0001F02DA7007221A710C225A719A799207B8
:10850000FCD59A79D006FCD40E4B19469A7902F024
:108510000C02082AFAD14C225A718B7903F00C0311
:10852000082BFAD1074B1A4699794906FCD5222126
:108530001970937903F00C030C2BFAD1704700BF2C
:1085400000700440004006400000330100001301A9
:1085500000500640264B5A7902F0E0025A711A790F
:1085600002F0F8021A71A3F500531A7802F08C0297
:1085700042F050021A705A7802F09C0242F0400217
:108580005A709A7802F0E6029A701A4A0023137021
:1085900083F31188184B012283F8182383F81923D9
:1085A000022283F8582383F8592383F81D2383F884
:1085B0001E2383F81F2383F8202383F8212303221B
:1085C00083F82D2383F82F2383F8312383F8332373
:1085D00083F83523042283F83923052283F83A23CC
:1085E000062283F85723072283F84923704700BFE8
:1085F00000F0074000E0074000E100E00C4A13688B
:10860000013313600B4A1368013313600A4B1A6875
:108610003AB11A68013A1A601B6813B9074B012274
:108620001A70074B1A6812B11A68013A1A6070473B
:108630001CC6FF1FF4CEFF1FECCCFF1FE8CCFF1FB2
:10864000F0CCFF1F024B034A5A6007221A607047A2
:1086500010E000E040190100014B1868704700BFAE
:108660001CC6FF1F1449154B41F23402072888BF6E
:10867000002010B553F82030114CB4FBF3F48B58A4
:1086800043F480638B500F4B4FF400725A602D20DF
:108690009A6006F05DF80C4B0022DA709A709A71BD
:1086A000DA725A71C4F30422E4B21A705C70DA7898
:1086B00042F02C02DA7010BD007004407414010006
:1086C00020AA44000090044000A00640094A136814
:1086D00051680133202B08BF00238B4208D011685A
:1086E000114408721360044AD37843F08003D370B6
:1086F000704700BF20C6FF1F00A006400A4B996AC2
:10870000DA6A91420DD09A6A511C1A44996292F821
:10871000302002709A6A202A01D100229A62012038
:1087200070470020704700BF20C6FF1F044B1A7817
:1087300002F0FF0012B100221A700120704700BF42
:10874000E8CCFF1F014B1865704700BF20C6FF1F14
:1087500030B526480179C9B28C0617D5244BDA6AA0
:108760009C6A0132202A08BF0022A2421BBFDC6A99
:10877000C579C27918191EBFEDB280F83050DA629F
:108780001C4A052010601A6D1B4B1A604A0608D55A
:108790001A4B4FF400329A60144AD37803F0BF03A7
:1087A000D3700B061BD5144B1868C0B9104B196851
:1087B0005A68914214D0114A4FF4003151605A68FE
:1087C000511C1A445960117A084AC9B2D1715968CA
:1087D000202908BF5860D37843F04003D37030BDE0
:1087E000024AD37803F07F03F8E700BF00A00640F9
:1087F00020C6FF1FECCCFF1FF0CCFF1F00F00F4086
:1088000062B67047FFF7FCBF72B67047FFF7FCBF58
:108810004FF0E02318B1034AC3F80C2D7047024A09
:10882000FAE700BF0400FA050100FA0510B9C9080B
:1088300001F07AB87047F7B5454A464E46494FF4BD
:108840008073136153619363D363136453647161E1
:10885000B160424940F20310086048608860C86017
:108860008862C8620B644B6401F5352140314FF4D6
:108870004030486148603A493A480B6040F6070486
:108880004B608B60CB624461446037480360436057
:108890008360C360036100F53320C0301424446159
:1088A0000424446010248460304C636104F5322455
:1088B00004F580742025656141F204042C4D2F5984
:1088C00027F0E0072F512F5947F0C0072F514FF4E1
:1088D000A064CC6013603446D360082600230A21CC
:1088E0001A46B4461F46A646C4F804C00197019D27
:1088F000B5F57A7F21D3DEF81050A660ED0748BFAA
:1089000001320197019DB5F57A7F1AD3DEF8105038
:10891000ED0758BF01330139E6D10A2A154A14D1AF
:108920000A2B12D101231370094B4FF4E0621A6035
:10893000DA601023436003B0F0BD019D013501955D
:10894000D5E7019D01350195DCE70023EBE700BF8A
:108950000090044000F00F402880030000A0044075
:1089600000B0044080F00F4000C0044000D004403C
:108970000070044028CDFF1FF7B5114B1B78E3B101
:1089800010491148114D20231E4600240F468646EB
:108990004E6086600194019AAA420AD9BB60CEF863
:1089A00004300194019AAA42F2D8019A013201924C
:1089B000F8E7019A01320192EDE703B0F0BD00BF84
:1089C00028CDFF1F00F00F4000F10F401FA107004E
:1089D000072809D8DFE800F004090C0F1114161855
:1089E0004FF400420A4B5A6070474FF48032F9E767
:1089F0000222084BF7E70822FBE74FF40062F8E792
:108A00000122F6E70422F4E74FF48062F1E700BFA9
:108A100000F00F4040F00F40072809D8DFE800F0D1
:108A200004090C0F111416184FF400420A4B9A60F7
:108A300070474FF48032F9E70222084BF7E708222B
:108A4000FBE74FF40062F8E70122F6E70422F4E7BF
:108A50004FF48062F1E700BF00F00F4040F00F409C
:108A600010B50021044644FA01F3DB07C8B205D56E
:108A7000FFF7AEFF01310829F5D110BDFFF7CCFF9C
:108A8000F8E708B506282CD8DFE800F0040D121727
:108A90001C212600002005F057FAB0F5806F34BF86
:108AA0000020012008BD104B186900F0010008BD2E
:108AB0000D4B1869C0F3800008BD0B4B1869C0F35B
:108AC000802008BD084B1869C0F3400008BD064B64
:108AD0001869C0F3C00008BD034B1869C0F3C0207B
:108AE00008BD002008BD00BF40F00F4007282DD86A
:108AF000DFE800F004090E13181D2227144B186834
:108B0000C0F3C0307047124B1868C0F30040704784
:108B1000104B1868C0F3400070470E4B1868C0F344
:108B2000C00070470B4B1868C0F3C0207047094B5A
:108B3000186800F001007047064B1868C0F3800009
:108B40007047044B1868C0F38020704700207047BE
:108B500000F00F4040F00F4070B50024254601267C
:108B6000E0B2FFF78EFF18B106FA04F31D43EDB231
:108B70000134082CF4D1284670BD10F0010F314BA0
:108B800033D05A6942F002025A614FF400329A60BF
:108B900010F0020F2C4A30D0596941F00801596198
:108BA0000221916041072FD5596941F40061596153
:108BB0004FF40061916001072ED5596941F0010120
:108BC00059614FF480319960C1062DD5596941F042
:108BD000040159610121916081062CD5596941F444
:108BE000806159610423936070474FF400325A60EA
:108BF0005A6922F002025A61CAE70221516059699A
:108C000021F008015961CDE74FF4006151605969C5
:108C100021F400615961CEE74FF480315960596900
:108C200021F001015961CFE701215160596921F01B
:108C300004015961D0E7042151605A6922F480622D
:108C40005A61704740F00F4080F00F401B4B5A684C
:108C500010F0010F14BF42F0030202F002025A604A
:108C6000DA6881074CBF42F0030202F00202DA60C8
:108C7000124BDA6A10F0040F14BF42F0030202F044
:108C80000202DA621A6801074CBF42F0030202F0E6
:108C900002021A60094B9A6810F0100F14BF42F0DC
:108CA000030202F002029A609A6A81064CBF42F007
:108CB000030202F002029A62704700BF00A0044063
:108CC00020B9034B1869C0F340307047002070474B
:108CD00000F00F4008B5082005F036F95E280DD9E0
:108CE0000F4B1A780AB901221A70082005F02CF9E6
:108CF00063280BD90B4B04229A6008BD082005F0AD
:108D000023F95428F1D80022054BEDE7082005F09F
:108D10001BF954289EBF034B04225A6008BD00BFB4
:108D200074C6FF1FC0F00F40034B187801380128AC
:108D30008CBF00200120704774C6FF1F034B1878BA
:108D4000012806BF02221A700020704774C6FF1F58
:108D5000C0B200F04FBFC0B200F040BF08B507F08E
:108D60000BFC05F0C9FE05F079FEBDE8084007F0F0
:108D700085BC38B5054605F0C7FD08280AD900248A
:108D80002819013405F040FE092CF9D105F070FED8
:108D9000012038BD002038BD092105F0D5BD0020D7
:108DA00006F062B82149224841F23C028B5843F454
:108DB00040538B501F4B012119601A6802431A60FF
:108DC0001D4ADA601A61DA6A42F08052DA621A6881
:108DD00022F001021A601A6822F000621A6003F59C
:108DE000F8334FF400721A615A619A61DA61A3F59F
:108DF000F03319601968014319601049D96001F511
:108E000020011961D96A41F08051D962196821F0B5
:108E100001011960196821F00061196003F5003340
:108E20001A605A609A60DA601A61704700700440F4
:108E3000000C1F8000C002400300013E0400513EB0
:108E4000FF281ED800041E4B00F47C108AB141F0AC
:108E5000006108435863DA6A002AFCDA184BDA6AC0
:108E6000D100FCD5986BDA6A42F01042C0B2DA62E7
:108E7000704741F0004108435863DA6A002AFCDA7F
:108E8000F0E7B0F5007F18D200040E4B00F47C1020
:108E90005AB141F0006108435863DA6A002AFCDAEB
:108EA000084BDA6AD200FCD5DCE741F00041084308
:108EB0005863DA6A002AFCDAD4E70020704700BF62
:108EC00000C0024000D00240C0EBC00038B5002214
:108ED0000C4600F5006503210120FFF7B1FF0022D9
:108EE000C5F307210120FFF7ABFF0022E9B2012003
:108EF000FFF7A6FF002211460120FFF7A1FF002285
:108F0000114620700120FFF79BFF00221146607080
:108F10000120FFF795FF00221146A0700120FFF706
:108F20008FFF00221146E0700120FFF789FF002229
:108F3000114620710120FFF783FF0122607100219B
:108F40001046FFF77DFFA07138BD38B54FF40064BF
:108F5000012206211046FFF773FF002205210120A0
:108F6000FFF76EFF012200211046FFF769FF80071F
:108F7000F3D5002202210120FFF762FF0022C4F393
:108F800007210120FFF75CFF0022E1B20120FFF77B
:108F900057FF0025A5F13F014A424A410120002127
:108FA0000135FFF74DFF402DF4D1002205210120AE
:108FB000FFF746FF012200211046FFF741FFC307DC
:108FC000F3D44034B4F5804FC2D138BDF7B5C0EB0F
:108FD000C00000F500650C46002203210120FFF7C8
:108FE0002FFFC5F3072100220120FFF729FFE9B277
:108FF00000220120FFF724FF002211460120FFF785
:109000001FFF0022114607460120FFF719FF00222B
:10901000114606460120FFF713FF002211460546C0
:109020000120FFF70DFF002211468DF803000120FB
:10903000FFF706FF002211468DF804000120FFF71C
:10904000FFFE01228DF8050000211046FFF7F8FE13
:1090500023788DF80600BB420ED16378B3420BD162
:10906000A378AB4208D1DDF80300D4F80330C31A6B
:109070005842584103B0F0BD0020FBE7012238B54B
:1090800004460D4610460621FFF7DAFE00220521B0
:109090000120FFF7D5FE012210460021FFF7D0FE88
:1090A0008207F3D5002202210120FFF7C9FE00222A
:1090B000C4F307210120FFF7C3FE0022E1B2012023
:1090C000FFF7BEFE012229461046FFF7B9FE002237
:1090D00005210120FFF7B4FE012200211046FFF711
:1090E000AFFEC307F3D438BD38B50D46C0EBC0049E
:1090F00004F500600978FFF7C1FF697804F6010004
:10910000FFF7BCFFA97804F60200FFF7B7FFE97884
:1091100004F60300FFF7B2FF297904F60400FFF715
:10912000ADFF697904F60500FFF7A8FFA97904F6F9
:109130000600BDE83840FFF7A1BF2DE9F843164609
:1091400001220446884610460621FFF779FE0022D8
:1091500005210120FFF774FE012200211046FFF7D0
:109160006FFE8507F3D5002202210120FFF768FE7C
:109170000022C4F307210120FFF762FE0022E1B2C2
:109180000120FFF75DFE0025771EB5420DD10022BC
:1091900005210120FFF754FE012200211046FFF7B0
:1091A0004FFEC307F3D4BDE8F883013414F03F0940
:1091B00018F8051039D0781B424242410120FFF7D0
:1091C0003FFEB9F1000F2ED1BD422CD20022052165
:1091D0000120FFF735FE012200211046FFF730FE87
:1091E000C107F3D4012206211046FFF729FE002211
:1091F00005210120FFF724FE012210460021FFF780
:109200001FFE8207F3D5002202210120FFF718FE7E
:109210000022C4F307210120FFF712FE0022E1B271
:109220000120FFF70DFE0135AFE70122C6E710B5BB
:109230000022044603210120FFF702FEC4F30721A8
:1092400000220120FFF7FCFDE1B200220120FFF720
:10925000F7FD012200211046BDE81040FFF7F0BDE8
:10926000F8B504460E461546032100220120FFF7FB
:10927000E7FDC4F3072100220120FFF7E1FDE1B281
:1092800000220120FFF7DCFD77193446013DBC4286
:1092900000D1F8BDA21BAB1A5A425A41002101204D
:1092A000FFF7CEFD04F8010BF1E737B500220521E9
:1092B0000120FFF7C5FD012200211046FFF7C0FD88
:1092C00010F07104F2D1FFF7C7F90546FFF7C4F9B2
:1092D000401B0028B8BF4042B0F5FA6F1DDA9CB1C0
:1092E000284B1B78DBB9402227490020FFF7B8FF45
:1092F000402210462549FFF7B3FF60222449254844
:1093000007F0D0F903B030BD40F2FF70FFF78FFFD8
:10931000A0F1AA035C425C41D8E7002CE0D1002117
:1093200040F2FF70FFF7AAFEFFF70FFE402216493A
:109330000020FFF702FF40221749104602ADFFF759
:10934000FCFE002345F8043D4FF4C364204604228C
:1093500029460434FFF7F1FEB4F5FF6FF6D1002380
:1093600001934FF4A7642046042229460434FFF7F2
:10937000E4FEB4F5C36FF6D1AA2140F2FF70FFF707
:109380007DFEB0E728CDFF1F0CC0FF1F44CDFF1F9F
:10939000A4140100ACCDFF1F0415010038B56FF017
:1093A000007204460D460C2105F012F80E212046ED
:1093B00005F034F82A466C21204605F009F80E2104
:1093C000204605F02BF88301F9D56E21204605F0E3
:1093D00025F8014B186038BD78C6FF1F38B5244CFE
:1093E000C300E2181179032984BF03211171E21827
:1093F0009179032984BF03219171E218117A0F2911
:1094000084BF0F211172E218517A072984BF072106
:109410005172E218917A0F2984BF0F219172E118DD
:109420000A794979D20342F40025E56011B142F48A
:109430000422E260E218D2791AB1E26842F40052E2
:10944000E26023441A7A9979D20142EAC122E168A2
:109450000A43597A42EA0112D97AE26011B99B7A39
:109460001A43E260E168FFF799FFE368236138BDC2
:1094700078C6FF1F10B5104C0023E360C300E2184C
:10948000527E12B14FF40072E260E218927E1AB17D
:10949000E26842F48072E260E2182344D17E0F2930
:1094A00084BF0F21D176D97EE3681943E160FFF7CD
:1094B00075FFE368E36110BD78C6FF1F38B5C200D1
:1094C0001F4C111A214491F8213091F8205091F845
:1094D00022101B0343EA853343F46025012908BFAA
:1094E0002B46A2EB000108BF43F480632144E560F2
:1094F00008BFE360E36891F8235091F8241043EA31
:1095000005230129E36004BF43F08003E360131ADD
:109510002344121A93F82530012B08BFE368224434
:1095200004BF43F04003E360E16892F8263041EA6B
:109530000311E160FFF732FFE368A36238BD00BFAB
:1095400078C6FF1F10B543001C4C1A18224492F92C
:109550002D103F29C4BF3F2182F82D101A18224434
:1095600092F92D103F31BCBFC12182F82D101A187D
:10957000224492F82E101F2984BF1F2182F82E103A
:109580004FF44022E2601A182244034492F82C203F
:109590002344012A04BF4FF45022E26093F82D10B7
:1095A000E26893F82E300902134301F4FE41194397
:1095B000E160FFF7F3FEE368236310BD78C6FF1F89
:1095C00010B58300244C1A18224492F83410012953
:1095D00084BF012182F834101A18224492F8351001
:1095E000032984BF032182F835101A18224492F807
:1095F00036100F2984BF0F2182F836101A18224422
:1096000092F83710032984BF032182F837101A1803
:109610002244034492F838100F29234484BF0F21B9
:1096200082F8381093F8381093F8342041F4202150
:1096300041EAC23193F8352041EA423193F83620AD
:1096400093F8373041EA022141EA4311E160FFF724
:10965000A5FEE368E36310BD78C6FF1F214B01211F
:109660001F2210B50520002483F82C1083F82E202B
:1096700083F82410032283F825100221197283F83D
:10968000261019715A729872DC7283F82D0083F8D3
:10969000202083F8212083F8224083F8234083F898
:1096A000344083F8354083F8364083F8374083F8F8
:1096B00038405C769C76DC765C71DC719C710A4B80
:1096C00004229A602046FFF77BFF2046FFF73AFF0F
:1096D0002046FFF7F3FE2046FFF7CCFE2046BDE80C
:1096E00010407BE678C6FF1FC0F00F40044B0429F2
:1096F00003EBC00318BF0022D97618BF5A76B9E62B
:1097000078C6FF1F034B03EBC003597609B104224F
:10971000DA76AFE678C6FF1F024B03EBC0039976FB
:10972000A8E600BF78C6FF1F024B03EBC000C07E57
:10973000704700BF78C6FF1F024B03EBC000407E9E
:10974000704700BF78C6FF1F024B03EBC000807E4E
:10975000704700BF78C6FF1F024B03EBC0031971AF
:109760003CE600BF78C6FF1F024B03EBC0035971F4
:1097700034E600BF78C6FF1F024B03EBC003D9716C
:109780002CE600BF78C6FF1F024B03EBC0039971A4
:1097900024E600BF78C6FF1F024B03EBC00319721B
:1097A0001CE600BF78C6FF1F024B03EBC0035972D3
:1097B00014E600BF78C6FF1F024B03EBC00399728B
:1097C0000CE600BF78C6FF1F024B03EBC000007918
:1097D000704700BF78C6FF1F024B03EBC000407903
:1097E000704700BF78C6FF1F024B03EBC000C07973
:1097F000704700BF78C6FF1F024B03EBC0008079A3
:10980000704700BF78C6FF1F024B03EBC000007A11
:10981000704700BF78C6FF1F024B03EBC000407AC1
:10982000704700BF78C6FF1F024B03EBC000807A71
:10983000704700BF78C6FF1F034B00EB8002134444
:1098400083F83410BCE600BF78C6FF1F034B00EB63
:109850008002134483F83510B2E600BF78C6FF1FBC
:10986000034B00EB8002134483F83610A8E600BFD8
:1098700078C6FF1F034B00EB8002134483F83710B8
:109880009EE600BF78C6FF1F034B00EB8002134427
:1098900083F8381094E600BF78C6FF1F034B00EB37
:1098A0008000184490F83400704700BF78C6FF1F4E
:1098B000034B00EB8000184490F83500704700BF60
:1098C00078C6FF1F034B00EB8000184490F8360069
:1098D000704700BF78C6FF1F034B00EB80001844A1
:1098E00090F83700704700BF78C6FF1F034B00EBAE
:1098F0008000184490F83800704700BF78C6FF1FFA
:10990000034B00EB4002134483F82C101AE600BF0F
:1099100078C6FF1F034B00EB4002134483F82D1061
:1099200010E600BF78C6FF1F034B00EB4002134454
:1099300083F82E1006E600BF78C6FF1F034B00EB2E
:109940004000184490F82C00704700BF78C6FF1FF5
:10995000034B00EB4000184490F92D00704700BF06
:1099600078C6FF1F034B00EB4000184490F82E0010
:10997000704700BF78C6FF1F034BC0EBC002134403
:1099800083F820109AE500BF78C6FF1F034BC0EB99
:10999000C002134483F8211090E500BF78C6FF1F72
:1099A000034BC0EBC002134483F8221086E500BFCE
:1099B00078C6FF1F034BC0EBC002134483F823108B
:1099C0007CE500BF78C6FF1F034BC0EBC002134409
:1099D00083F8241072E500BF78C6FF1F034BC0EB6D
:1099E000C002134483F8251068E500BF78C6FF1F46
:1099F000034BC0EBC002134483F826105EE500BFA2
:109A000078C6FF1F034BC0EBC000184490F820003D
:109A1000704700BF78C6FF1F034BC0EBC00018445F
:109A200090F82100704700BF78C6FF1F034BC0EBC2
:109A3000C000184490F82200704700BF78C6FF1F8E
:109A4000034BC0EBC000184490F82300704700BFE0
:109A500078C6FF1F034BC0EBC000184490F82400E9
:109A6000704700BF78C6FF1F034BC0EBC00018440F
:109A700090F82500704700BF78C6FF1F034BC0EB6E
:109A8000C000184490F82600704700BF78C6FF1F3A
:109A90002DE9F0479046334A089F099E1D4613184A
:109AA000044693F8403089469246042B2FD8DFE8CD
:109AB00003F0031A20262C00FFF790FC0AEB0403A6
:109AC0000122C4EBC404544483F8402094F82630A7
:109AD000012B31D01FD3022B35D016B1DAF800306C
:109AE0003370BDE8F087FFF7E9FC0AEB04030222BC
:109AF000E7E7FFF765FD0AEB04030322E1E7FFF761
:109B000021FD0AEB04030422DBE7FFF7B3FC0AEBB9
:109B100004030022D5E7B9F1000F04D0DAF80030D1
:109B20009B0C89F80030B8F1000FD6D0DAF800307D
:109B30009B0A88F80030D0E7002DCED0DAF800304C
:109B40009B0A2B60C9E725B1DAF80030DB0B5B011B
:109B50002B60002FC1D0DAF80030C3F384233B70B0
:109B6000BBE700BF78C6FF1F2DE9F84388466C218C
:109B700005461C469146089F099E04F04FFC164B73
:109B8000C5EBC5051D4495F82630012B14D005D32F
:109B9000022B16D006B13070BDE8F883B8F1000F83
:109BA00002D0830C88F80030B9F1000FF2D0C0F376
:109BB0008923A9F80030EDE7002CEBD0830A23605D
:109BC000E8E714B1C30B5B012360002FE2D0C0F3C0
:109BD00084233B70DEE700BF78C6FF1F30B9044B1B
:109BE000DA7A1AB90122DA72FFF7F8BB704700BFC0
:109BF00078C6FF1F28B9034BD97A11B1D872FFF785
:109C0000EDBB704778C6FF1F062808D8DFE800F0D4
:109C100004080B0E111417000A4B1B680B607047E9
:109C2000084BDB69FAE7074B1B69F7E7054BDB6B72
:109C3000F4E7044B1B6BF1E7024B9B6AEEE7014B29
:109C4000DB7AEBE778C6FF1F044B9A78044B12B11E
:109C500004221A7070470322FBE700BF84CEFF1F67
:109C6000F8CEFF1F38B5044CA278637842B1034B9D
:109C700004221A7038BD00BF84CEFF1FF8CEFF1F2C
:109C8000FF2B00F2FD83DFE813F0A001B501C8014E
:109C9000D201DD01E401E901EE01F301FC01020260
:109CA0000B021402280251025602600265026A0287
:109CB00074027902830288028F0296029D02A40236
:109CC000AB02B202C602FB03FB03FB03CF02DB02C3
:109CD000FB03FB03FB03FB03FB03FB03FB03FB0394
:109CE000FB03FB03FB03FB03FB03FB03FB03E2029E
:109CF000FB03FB03FB03FB03FB03FB03FB03FB0374
:109D0000FB03FB03FB03FB03FB03FB03FB03FB0363
:109D1000FB03FB03FB03FB03FB03FB03FB03FB0353
:109D2000FB03FB03FB03FB03FB03FB03FB03FB0343
:109D3000FB03FB03FB03FB03FB03FB03FB03FB0333
:109D4000FB03FB03FB03FB03FB03FB03FB03FB0323
:109D5000FB03FB03FB03FB03FB03FB03FB03FB0313
:109D6000FB03E802ED02F202F702FC020103060324
:109D70000B03100315031A031F0324032903FB031A
:109D80002E0335033A033F03440349035003FB0307
:109D900055035C0363036903FB036E0374038303CE
:109DA000FB038803FB03FB03FB03FB03FB03FB0336
:109DB000FB03FB03FB03FB03FB03FB03FB03FB03B3
:109DC000FB03FB03FB03FB03FB03000115011B016A
:109DD000210127012D01330139013F0145014B01CB
:109DE000510157015C01620168016E0174017A0141
:109DF000800186018B01900195019A01FB03FB0311
:109E0000FB03FB03FB03FB03FB03FB03930398032D
:109E1000A003A803AD03FB03FB03B203B703BD0319
:109E2000FB03FB03FB03C203FB03C703CC03D80301
:109E3000FB03DD03E203E703FB03FB03FB03FB037D
:109E4000FB03FB03FB03FB03FB03FB03FB03FB0322
:109E5000FB03FB03FB03FB03FB03FB03FB03FB0312
:109E6000FB03FB03FB03FB03FB03FB03FB03FB0302
:109E7000FB03FB03FB03FB03FB03FB03FB03FB03F2
:109E8000FB03FB03EC03F103F6030020FFF754FC94
:109E90009C4B58609C4B1B785BB19A4B5A689B4B10
:109EA0001A609B4B002A40F0EF821A6842F00802C9
:109EB0001A6038BD0020FFF747FC924B5860E9E775
:109EC0000020FFF781FC8F4B5860E3E70020FFF78D
:109ED00083FC8C4B5860DDE70020FFF78DFC894B3D
:109EE0005860D7E70020FFF78FFC864B5860D1E71A
:109EF0000020FFF791FC834B5860CBE70020FFF771
:109F000093FC804B5860C5E70020FFF7C7FC7D4BF2
:109F10005860BFE70020FFF7CBFC7A4B5860B9E7E9
:109F20000020FFF7CFFC774B5860B3E70020FFF726
:109F3000D3FC744B5860ADE7764B5A79714B5A603D
:109F4000A8E70020FFF7FAFC6E4B5860A2E700205C
:109F5000FFF7FEFC6B4B58609CE70020FFF752FDBB
:109F6000684B586096E70020FFF756FD654B586038
:109F700090E70020FFF75AFD624B58608AE7002007
:109F8000FFF75EFD5F4B586084E70020FFF76CFD34
:109F90005C4B58607EE7604B1A785A4B5A6079E701
:109FA0005E4B1A69574B5A6074E75A4B1A68554B07
:109FB0005A606FE7574B1A79524B5A606AE7002094
:109FC000FFF712FC4F4B586064E7002003F048F99C
:109FD0004C4D372120B9A07804F020FA686059E789
:109FE000A07804F01BFAA2784D4B53F82230C01A27
:109FF00068604FE74B4B434D1878212118B904F0A6
:10A000000DFA686046E7002004F008FAA278444B95
:10A0100053F82230C01A68603CE7434B24210020EB
:10A020001C6804F0FBF9A047364B586032E73E4B02
:10A03000222100201C6804F0F1F90002A047314BF6
:10A04000586027E7384B1A68586890472D4B58607E
:10A0500020E7324B9A6A2B4B5A601BE72F4B5A7AF8
:10A06000284B5A6016E72D4B9A7A264B5A6011E717
:10A070000F21002004F0D2F9224B00F001005860BB
:10A0800008E7002004F03CFB1E4B586002E70F215C
:10A09000002004F0C3F91B4BC0F300205860F9E620
:10A0A0000F21002004F0BAF9164BC0F3C01058601D
:10A0B000F0E60121002004F0B1F9830741BF114A05
:10A0C000536843F00103536005077FF5E3AE0D4A83
:10A0D000536843F002035360DCE60121002004F0E2
:10A0E0009DF9C40741BF074A536843F00103536019
:10A0F00041077FF5CFAE034A536843F00203536034
:10A10000C8E600BFF8CEFF1FF3CEFF1FE4CEFF1F4F
:10A110008CCEFF1F10CDFF1F0CCDFF1F44CDFF1FA6
:10A1200008CDFF1FACCDFF1FBCC6FF1F944BDA7DCF
:10A13000944B5A60AEE6944B252100201C6804F035
:10A140006DF9A0478F4B5860A4E68D4B1A6B8D4B71
:10A150005A609FE68A4BDA6A8A4B5A609AE68A4BC3
:10A16000272100201C6804F059F9A047854B58604E
:10A1700090E6834B5A6B834B5A608BE6824B2621C9
:10A1800000201C6804F04AF9A0477E4B586081E625
:10A190007B4B9A6B7B4B5A607CE62D21002004F0B0
:10A1A0003DF9784B586075E62E21002004F036F911
:10A1B000744B58606EE62F21002004F02FF9714B8C
:10A1C000586067E63021002004F028F96D4B586094
:10A1D00060E63321002004F021F96A4B586059E60B
:10A1E0003421002004F01AF9664B586052E6012130
:10A1F000002004F013F9420641BF624A536843F05D
:10A200000103536003067FF545AE5E4A536843F091
:10A21000020353603EE60121002004F0FFF8594B91
:10A22000C0F30120586035E60121002004F0F6F863
:10A2300010F0100F534B14BF012200225A6029E680
:10A240000121002004F0EAF810F0200FF2E70020CE
:10A2500003F074FB4B4B58601CE64C4B5A68494B5F
:10A260005A6017E6494B9A68464B5A6012E6474BCC
:10A270001A7B444B5A600DE6444BDA89414B5A60D5
:10A2800008E6424B1A693F4B5A6003E63F4B1A7D82
:10A290003C4B5A60FEE53D4B5A7D3A4B5A60F9E51E
:10A2A0003A4B1A6A374B5A60F4E5384B5A6A354BC9
:10A2B0005A60EFE5354B9A6A324B5A60EAE5334B08
:10A2C000DA6A304B5A60E5E5304B1A6B2D4B5A6019
:10A2D000E0E52E4B9A692B4B5A60DBE52B4BDA6994
:10A2E000284B5A60D6E57C21002004F097F8254BD6
:10A2F0005860CFE5254B5A6B224B5A60CAE5234B79
:10A300009A6B204B5A60C5E5204B9A7D1D4B5A60D5
:10A31000C0E51D4B1A7A1B4B5A60BBE5202100207B
:10A3200004F07CF8174B5860B4E5184B1A78154BBD
:10A330005A60AFE56621002004F070F8114B5860B8
:10A34000A8E56521002004F069F80E4B5860A1E5EE
:10A35000002002F085FF0B4B58609BE50B4BDA6B3E
:10A36000084B5A6096E5094B93F84020054B5A601C
:10A3700090E5064B93F84120024B5A608AE500BFF6
:10A3800044CDFF1FF8CEFF1FBCC6FF1FACCDFF1F83
:10A390003F4B5A6C3F4B5A607CE50A21002004F089
:10A3A0003DF83C4B00F00F00C0F10800586071E52B
:10A3B000394B1A7A374B5A606CE5374A374B10687D
:10A3C0001B689847334B586064E5334A334B5068F9
:10A3D0001B6898472F4B58605CE5314B1A682D4B32
:10A3E0005A6057E52F4B1A682A4B5A6052E52A4BA0
:10A3F0009A7D284B5A604DE5002003F093FF254BD2
:10A40000586047E5244B9A8F224B5A6042E5264B11
:10A410001A68204B5A603DE5244B1A781D4B5A6050
:10A4200038E55021002003F0F9FFA278204B53F8C3
:10A430002230C01A174B58602CE5174BDA69154BC0
:10A440005A6027E5144B1A6A124B5A6022E5124BE8
:10A450005A6A104B5A601DE50F4B9A8A0D4B5A6091
:10A4600018E5144B1A680B4B5A6013E50A4B5A7ED9
:10A47000084B5A600EE5084B1A7E064B5A6009E5F8
:10A48000044B03221A7005E51A6822F008020FE552
:10A49000ACCDFF1FF8CEFF1F44CDFF1FBCC6FF1F72
:10A4A000FCCCFF1F0CCEFF1F24CDFF1F41CDFF1F93
:10A4B0001CCDFF1F30CDFF1F38B5B24A9378022B59
:10A4C000144600F00681032B00F00A81002B40F0B7
:10A4D000738153784E2B00F0B38030D8462B00F0B8
:10A4E000818012D8422B6DD006D8402B5ED0412BF4
:10A4F00063D00322A44B57E0442B68D0452BF8D1FE
:10A50000A24BD1785971052053E04B2B00F0888085
:10A510000BD8472B6ED0492BEBD1D2789B4B002A1E
:10A5200079D1DA75D97D172043E04C2B00F0838078
:10A530004D2BDED1954BD1785975152039E0542B30
:10A5400000F0A5801BD8512B00F08C8009D84F2B30
:10A5500000F08180502BCCD18C4BD178997516208E
:10A5600027E0522B00F08B80532BC2D1874DD2F8BD
:10A5700003302946042241F8103F102042E0842B8A
:10A5800000F09D8009D8552B00F08D80832BB0D131
:10A590007F4BD2F80320DA6038BD852B00F0948021
:10A5A000FF2BA6D1D2787B4B1A70B5E0D17840F260
:10A5B000FF70BDE83840FEF761BD744BD17819706B
:10A5C0000020F6E7714BD17859700120F1E76F490F
:10A5D000D2F8033041F81C3F04221C20BDE838406B
:10A5E000FEF7ABBD6949D2F8033041F80C3F0422B5
:10A5F0000C20F3E7654DD2F803302946042241F8D8
:10A60000083F0820FEF799FD2A8A29896879BDE864
:10A61000384003F0CBBC5C490122DA754A6081E71F
:10A620005A4CD178E1700320FEF728FDE078BDE8B0
:10A630003840FEF787B8554BD17899700220B8E7BB
:10A64000524CD2F80300E084FEF797FA022204F19C
:10A6500026012620C2E7D2F803104C4BC9B2597626
:10A660001920A6E7494D2A7DD20704D5E378DB07F8
:10A6700001D4FEF76AFCE1782975142099E7434973
:10A68000D2F8033041F8203F04222020A6E7D2F878
:10A690000330012B00F290803C49D37801F81A3F37
:10A6A00001221A209AE7D2F80330012B00F28480AD
:10A6B0003649D37801F81B3F01221B208EE7364B29
:10A6C000D2F803201A6038BDD2F80320304B1A614B
:10A6D00038BD5178314BD2F8032043F8212038BDE2
:10A6E0005378272B41D018D8022B35D00CD853B330
:10A6F000012B7FF4FEAE2A4BD2F803205A60FDF7FF
:10A70000ABFF234B986138BD092B05D0FFF4F1AEA8
:10A710001B3B012B3FF6EDAE38BD2B2B2DD007D8C0
:10A72000292BD2F803201E4B25D022D9DA6138BD5F
:10A730002D2B3CD036D32E2B7FF4DBAE184BD2F82A
:10A740000320DA6238BD164BD2F803201A60FDF7F9
:10A7500083FF0F4B586138BD114BD2F803209A602C
:10A76000FDF77AFF0A4BD86138BDD2F803200C4BB5
:10A77000ADE75A6138BD9A6138BD094BD2F8032064
:10A780001A6238BD84CEFF1FF8CEFF1F0CC0FF1F1A
:10A79000BCC6FF1FF2CEFF1FF4CEFF1F04CFFF1F6A
:10A7A00010CEFF1F054BD2F803205A6238BD034B71
:10A7B000D2F803209A6238BD04229BE610CEFF1F18
:10A7C000404B2DE9F04100251D603F4B3F4C1D6083
:10A7D0003F4B2562284624211D6084F8245003F055
:10A7E0001DFE3C4B60601D703B4D2B7E002B40D10D
:10A7F0003A4BA3622360E362236328210020266B87
:10A8000003F00CFEB0472921A8620020266B03F05C
:10A8100005FEB0472A21E8620020266B03F0FEFD0A
:10A82000B0472B2128630020266B03F0F7FDB047CB
:10A830002C2168630020266B03F0F0FDB047284A06
:10A84000A86300231946174642F823100133B3F5D5
:10A85000807FF9D1234EB27E9AB9F37E0BB3737D1C
:10A860006BB3FEF761FA50B3012384F83430BDE8CE
:10A87000F0811D4BA3621D4B23601D4BE3621D4BFA
:10A88000BAE7DFF874804FF4C365A5F21461284677
:10A89000042241440435FEF7E3FCB5F5CD6FF4D155
:10A8A000DBE74FF4A765A5F5A761284604223944E4
:10A8B0000435FEF7D5FCB5F5C36FF4D1CFE700231F
:10A8C000D3E700BFE4CEFF1F00CFFF1FBCC6FF1FB2
:10A8D0008CCEFF1F19CDFF1F44CDFF1F1FE70000C7
:10A8E00004CFFF1F0CC0FF1F0FE7000017E7000099
:10A8F00013E700001BE7000090CEFF1F014B93F809
:10A9000035007047BCC6FF1F70B55B4E5B4B6425BE
:10A9100005FB00650446A96A99420BD8EA6A9A4287
:10A9200008D82A6B9A4205D86A6B9A4202D8AA6B59
:10A930009A4272D9642505FB046502220021204653
:10A9400003F0ACFDA86A06F0EFFB06F0A9F80022C0
:10A950004B4B06F0F9F846A3D3E9002306F01EFAA4
:10A9600006F004FB28210246204603F031FDE86A88
:10A9700006F0DAFB06F094F80022414B06F0E4F80A
:10A980003BA3D3E9002306F009FA06F0EFFA2921E8
:10A990000246204603F01CFD286B06F0C5FB06F0BE
:10A9A0007FF80022364B06F0CFF831A3D3E900231D
:10A9B00006F0F4F906F0DAFA2A210246204603F0FE
:10A9C00007FD686B06F0B0FB06F06AF800222C4B1E
:10A9D00006F0BAF826A3D3E9002306F0DFF906F063
:10A9E000C5FA2B210246204603F0F2FCA86B06F0C4
:10A9F0009BFB06F055F80022214B06F0A5F81CA39E
:10AA0000D3E9002306F0CAF906F0B0FA02462C2179
:10AA10002046BDE8704003F0DBBC1A4E06EB84060E
:10AA20000222002103F048FDF36AA86A9847282112
:10AA30000246204603F0CCFCF36AE86A98472921D5
:10AA40000246204603F0C4FCF36A286B98472A218B
:10AA50000246204603F0BCFCF36A686B98472B2142
:10AA60000246204603F0B4FCF36AA86B9847CDE792
:10AA7000000000A2941AED4244CDFF1FFFFF3F00EB
:10AA800000004042BCC6FF1F73B5034CA278637838
:10AA900022B1042200F06BBC84CEFF1FFF2B00F21A
:10AAA000F784DFE813F0D901EA0106021102190266
:10AAB00034023E025402F504F504F504F504600284
:10AAC000730284028C02940299029E02A602AB02D7
:10AAD000B302B802BC02C002C402C802CC02D00257
:10AAE000EF02F504F504F504FC020A03F504F5048D
:10AAF000F504F504F504F504F504F504F504F5048E
:10AB0000F504F504F504F504F5041803F504F5045B
:10AB1000F504F504F504F504F504F504F504F5046D
:10AB2000F504F504F504F504F504F504F504F5045D
:10AB3000F504F504F504F504F504F504F504F5044D
:10AB4000F504F504F504F504F504F504F504F5043D
:10AB5000F504F504F504F504F504F504F504F5042D
:10AB6000F504F504F504F504F504F504F504F5041D
:10AB7000F504F504F504F504F504F504F5042503DE
:10AB80002B033103410351035703640375037B0314
:10AB900081038F039B03A103A703F504F504AD0311
:10ABA000B303B903C403CD03D103F504F504F504DD
:10ABB000F504DB03F504E103EF03F903F5040004F6
:10ABC000F504F504F504F504F504F504F504F504BD
:10ABD000F504F504F504F504F504F504F504F504AD
:10ABE000F504F504F5040001090112011B0124011B
:10ABF0002D0136013F01480151015A0163016C01E9
:10AC00007B0184018D0196019F01A801B101F5042A
:10AC1000BA01BF01CB01D001F504F504F504F50438
:10AC2000F504F504F504F504120416041E04F504F5
:10AC3000F504F504F504260430043804F504F5049D
:10AC4000F504F504F504F50471049104F504B40465
:10AC5000BA04BF04F504F504F504F504F504F5049D
:10AC6000F504F504F504F504F504F504F504F5041C
:10AC7000F504F504F504F504F504F504F504F5040C
:10AC8000F504F504F504F504F504F504F504F504FC
:10AC9000F504F504F504F504F504F504F504F504EC
:10ACA000C704CD04DB04D4F803100020C9B202B0FD
:10ACB000BDE87040FEF726BDD4F803100020C9B2ED
:10ACC00002B0BDE87040FEF727BDD4F803100020A5
:10ACD000C9B202B0BDE87040FEF73EBDD4F8031023
:10ACE0000020C9B202B0BDE87040FEF73DBDD4F807
:10ACF00003100020C9B202B0BDE87040FEF744BDA9
:10AD0000D4F803100020C9B202B0BDE87040FEF7CD
:10AD100043BDD4F803100020C9B202B0BDE87040B2
:10AD2000FEF742BDD4F803100020C9B202B0BDE85E
:10AD30007040FEF741BDD4F803100020C9B202B044
:10AD4000BDE87040FEF778BDD4F803100020C9B20A
:10AD500002B0BDE87040FEF779BDD4F803100020C2
:10AD6000C9B202B0BDE87040FEF77ABDD4F8031056
:10AD70000020C9B202B0BDE87040FEF77BBDD4F838
:10AD800003100020C9B2FEF77FFDA278B64B03EB9B
:10AD9000C203D4F803205A7102B070BDD4F8031076
:10ADA0000020C9B202B0BDE87040FEF7A9BDD4F8DA
:10ADB0000310002049B202B0BDE87040FEF7AABD02
:10ADC000D4F803100020C9B202B0BDE87040FEF70D
:10ADD000D3BDD4F803100020C9B202B0BDE8704062
:10ADE000FEF7D4BDD4F803100020C9B202B0BDE80C
:10ADF0007040FEF7D5BDD4F803100020C9B202B0F0
:10AE0000BDE87040FEF7D6BDD4F803100020C9B2EB
:10AE100002B0BDE87040FEF7E1BD944BD4F80320CA
:10AE20001A61B9E7D4F803008F4B18600028B3D13A
:10AE3000597902B0BDE87040FEF726BD8A4BD4F8C0
:10AE400003201A71A8E7D4F803100020C9B202B099
:10AE5000BDE87040FEF790BC854BD4F8032018780D
:10AE600028B9372102B0BDE8704003F0B1BA814B78
:10AE70001B6837211A440020F4E77D4B187818B975
:10AE8000D4F803202121EDE72121002003F0C6FAA8
:10AE9000D4F80330A578C01A764B502118602846A4
:10AEA00003F0BCFAD4F80330C01A734B43F8250002
:10AEB00072E7724BD4F8030001221A70704B9B6A40
:10AEC000984724210246D6E76D4BD4F803009B6ACD
:10AED000984722210246CEE7694DD4F80300AB6AB9
:10AEE00098470028B8BF404268602021A07803F04E
:10AEF00095FA40077FF550AFA678D4F8030005EB2C
:10AF00008605AB6A9847242102463046AAE7574B8C
:10AF1000D4F803209A62002002B0BDE87040FFF729
:10AF2000F3BC534B51481B78E178417243B9827AA4
:10AF3000807D019000911846062103F01FFA2BE74F
:10AF4000C908002002B0BDE87040FEF7EDBC484BD8
:10AF500046491B78E2788A72002B7FF41DAF887D0A
:10AF60000190497AE6E70121002003F057FAD4F86E
:10AF7000033020F00A02D90748BF42F002029E07C0
:10AF800001D542F008020121A0786BE701210020E1
:10AF900003F044FAD4F8033020F00502DD0748BF7F
:10AFA00042F001029807EED542F00402EBE7D4F834
:10AFB0000330012B3FF66DAD2C4AD375ECE6304BD8
:10AFC000D4F803009B6A98472521024653E7274B94
:10AFD000D4F803201A639EE7244BD4F80320DA62E6
:10AFE00099E7274BD4F803009B6A9847272102462C
:10AFF00041E71E4BD4F803205A638CE7204BD4F86A
:10B0000003009B6A98472621024634E7174BD4F881
:10B0100003209A637FE7D4F803202D212BE7D4F88F
:10B0200003202E2127E7D4F803202F2123E7D4F88B
:10B03000032030211FE7D4F8032033211BE7D4F885
:10B040000320342117E70121002003F0E7F9D4F8A9
:10B05000033020F0C002D90748BF42F040029B07EE
:10B0600091D542F080028EE710CDFF1F44CDFF1F27
:10B07000ACCDFF1F08CDFF1F1CCDFF1F19CDFF1F3B
:10B08000BCC6FF1F0121002003F0C8F9D4F803302B
:10B090001B0220F4407203F440731A4373E701214A
:10B0A000002003F0BBF9D4F8033020F01002002B8D
:10B0B0003FF469AF42F0100265E70121002003F080
:10B0C000ADF9D4F8033020F02002002B3FF45BAF41
:10B0D00042F0200257E7A74B1B78002B3FF45CAEF1
:10B0E000D4F80310002002B0BDE8704002F008B9A7
:10B0F000A04BD4F803205A606021BCE69D4BD4F8E5
:10B1000003209A606121B6E69A4BD4F803201A73A3
:10B110001C21002003F082F9D4F80320C0F30800BA
:10B1200040EA02421C212FE7924BD4F80320DA8137
:10B130001C21002003F072F9D4F8033000F47F02E0
:10B14000C3F308031A43EDE78A4BD4F803201A61CE
:10B15000592190E6874AD4F803101378C9B21175C3
:10B16000002B3FF419AE937D0191527D0BE0814994
:10B17000D4F803200B78D2B24A75002B3FF40CAE02
:10B180008B7D097D01910092062100220020D4E6EA
:10B19000784BD4F803201A625A216CE6754BD4F828
:10B1A00003205A625B2166E6D4F80320714BD1B2CA
:10B1B0009A62C2F3072293F82C3001910092002288
:10B1C0005D21E3E76B4AD4F80330D362926AD1B2CF
:10B1D000C2F3072201910092DBB2F0E7654BD4F88D
:10B1E00003201A635E2146E6624BD4F803209A617D
:10B1F000182140E65F4BD4F80320DA6119213AE6C2
:10B200005C4BD4F803205A635C2134E6594BD4F8E4
:10B2100003209A635F212EE6564AD4F80330117852
:10B22000DBB2937500293FF4B7AD117D9CE7D4F8EC
:10B230000330022B3FF62DACE2784F4B1A72ABE590
:10B24000D4F80320202116E6D4F80330494A012B14
:10B250000ABF4A4900230B7013709DE5454BD4F893
:10B260000320DA63522106E6424BE1785A6C83F8F8
:10B270004010019193F841300093D3B26321C2F39F
:10B28000072283E73B4BE17883F841105A6C93F82F
:10B2900040308DE80A00F0E7364BD4F803205A64BA
:10B2A00093F84010E5E7D4F80330082B3FF6F1ABF4
:10B2B0000A21002003F0B2F8D4F8033020F00F0286
:10B2C000C3F108031A430A215EE6D4F803202C4B8D
:10B2D000B4E7294BD4F803009B6A9847284B1860C1
:10B2E0005AE5254BD4F803009B6A9847244B5860D5
:10B2F00052E5204B22491B78E0788875002B7FF4BB
:10B300004BAD8A7A2CE6D4F80310002002B0BDE8D9
:10B31000704002F0BFBF1A4ED4F80320B38F9A4298
:10B320003FF43AAD134B187800BB0C23B2870A21C7
:10B33000009392B2042303F0CDF8A078642505FBB6
:10B3400000635421DA69002AB8BF524203F040F882
:10B35000A07805FB00654FF00052EB690721002B38
:10B3600050DA02B0BDE8704003F098B80622054BF1
:10B370001A7011E5ACCDFF1FBCC6FF1F19CDFF1F12
:10B3800044CDFF1FF8CEFF1F424B434E1D788DB1B9
:10B390005021002003F042F8D4F80330A578C01AF9
:10B3A00030602121284603F039F8D4F80330C01A60
:10B3B0003A4B7BE5D4F803205021284603F008F8E7
:10B3C000A37846F82350E7E4354DD4F80320EB6921
:10B3D0009A423FF4E1AC2F4B18780028C6D1002ADE
:10B3E000B8BF5242542102F0F3FFA078D4F80320F2
:10B3F000642303FB0053002ADA614FF007014FF08A
:10B400000052ADE702B0BDE8704003F055B8244BE0
:10B41000D4F803201A6253212DE5214BD4F80320E0
:10B420005A62B9E41E4AD4F8033093821D4A1521AA
:10B430005A4320E51C4BD4F803201A6012211AE568
:10B44000D4F803300F2B3FF624ABE178144B0020E7
:10B45000597602B0BDE8704001F00ABFD4F803305D
:10B460006BB1012B7FF415AB0D4A13760F4B104ACD
:10B470009A62104A1A60104ADA62104A06E0084AD4
:10B4800013760A4B0E4A9A621A60DA621A6383E4F0
:10B4900003226CE7ACCDFF1F1CCDFF1F08CDFF1FA3
:10B4A00044CDFF1F0071020030CDFF1FBCC6FF1F3F
:10B4B0000FE7000017E7000013E700001BE700009C
:10B4C0001FE700002DE9F341C14EDFF838833278E1
:10B4D000D6F8033088F801206427212A88F8007004
:10B4E000C8F804303446454600F0C28700F2B980FF
:10B4F0000E2A00F0EE843AD8072A00F07B8314D895
:10B50000032A00F0118208D8012A00F09081022A53
:10B5100000F0CE8102232B70C2E1052A00F0678380
:10B5200040F21E82FEF79EFBBAE10A2A00F0688311
:10B5300007D8082A00F06183092AEBD1FEF7BCFF87
:10B54000AEE10C2A00F0968440F27E84B0780028A8
:10B5500040F0AB817378012B00F0A284C0F09D8491
:10B56000022B00F0A084032388F8003098E1182A09
:10B5700000F0E6852BD8142A00F0348515D80F2A60
:10B5800000F0CC84132AC5D17178924A092900F2BF
:10B59000FF84DFE811F0FA04050508050B050F0527
:10B5A000160519051C051F051405162A00F0C4858B
:10B5B00040F23785884A916B072900F27181481C57
:10B5C00002EB81019063106AC863136268E11C2A70
:10B5D00000F0A28620D81A2A00F0D08540F2BD855E
:10B5E0007D4D95F8242062B95A1C04BF794B1B6825
:10B5F0000A2058432866FDF72FF80123686685F86E
:10B6000024306378042B00F24B81DFE813F0C80587
:10B6100004062F065A06DC051F2A00F0A88600F251
:10B62000E5861E2A7FF476AF7078142800F21B841A
:10B63000B278002A40F07C86684941F82030684B97
:10B640009B7E002B00F02C81002800F0298100F265
:10B6500085108000A0F2146304221944FDF76DFDEB
:10B660001EE1802A00F0EE8741D8402A00F0D28700
:10B6700026D8242A00F05A870CD8222A00F04E87B8
:10B68000232A7FF447AF534B1B68C6F80330FEF7FD
:10B6900013FF05E1262A00F09787C0F07A87272A52
:10B6A0007FF438AFB378002B40F0FF807378142B11
:10B6B00000F2D983474A1168484A42F82310EFE064
:10B6C000442A00F0B38707D8422A00F0AB8740F243
:10B6D000A58701F0C0FDE3E0462A00F0AF87C0F087
:10B6E000A987472A7FF416AF01F0B9FDD8E0872A71
:10B6F00001F04A8047D8832A00F0C4870AD8812AFB
:10B7000000F0A687822A7FF405AF334B022283F82C
:10B710003420C5E0852A00F0EA87314A40F2D2871A
:10B720003049314C01250D709178217040F2FE7145
:10B730008B4200F2E287127D12EA050640F0DD87B7
:10B7400018466946FDF7C0FB9DF8003063709DF810
:10B750000130A3709DF80230E3709DF8063023712C
:10B760009DF8053063719DF80430A3719DF8033096
:10B77000E37126722B46E15C227A01330A44082BDE
:10B780002272F8D18CE08C2A01F050803CD8892AB2
:10B7900001F03180C0F0BB878A2A7FF4BBAE72789B
:10B7A000124B002A41F03F801A70114AE37813705F
:10B7B000094A92F84C110F4A11700F4900220A7081
:10B7C0000E490A700E4A11780B43137068E000BFEF
:10B7D00084CEFF1FE4CEFF1FBCC6FF1F90CEFF1F0D
:10B7E0000CC0FF1FE8CEFF1FE9CEFF1F00CDFF1FDB
:10B7F00020CDFF1F4ECEFF1F1ACDFF1F81CEFF1F92
:10B8000001CDFF1FF8CEFF1FF22A01F09B80FF2A17
:10B8100001F0DD808D2A7FF47DAE7278032A01F27B
:10B820008C80DFE812F047082E0877088508B37887
:10B83000002B3AD1002001F091FD0125B078B74BE3
:10B840004FF0006229461D5402F028FEB078B44A39
:10B85000642303FB0023DB7D2BBB2A46202102F05F
:10B86000B7FDA578AF4BD4F8030003EB85039B6AC3
:10B87000984724210246284602F0AAFD4FF0805244
:10B880000721A07802F00AFE4FF000620721A0789D
:10B8900002F012FE4FF000620121A07802F00CFECF
:10B8A00002B0BDE8F0810222D8E704232B70F7E74D
:10B8B000B0780028F9D101F051FD0125B078974BFF
:10B8C0004FF0006229461D5402F0E8FDB078944A1A
:10B8D000642303FB0023DB7D23BB2A46202102F0E7
:10B8E00077FDA5788F4BD4F8030003EB8503404226
:10B8F0009B6A984724210246284602F069FDA078F9
:10B900004FF08052072102F0C9FDA0784FF000628D
:10B91000072102F0D1FD4FF000620121A07802F072
:10B92000CBFDBDE70222D9E7B0780028BDD102F0F7
:10B93000B9FAB078794B01221A54794B07FB0037DA
:10B94000FB7D5BB9202102F043FDA0780022242179
:10B9500002F03EFDA07801F001FDA1E70222F1E72F
:10B96000B07810B17278022A9AD16678012E00F070
:10B9700087803FD3022E93D1142B96DC020640F130
:10B98000EE80C3078CD5002001F0E8FC644BD87D25
:10B99000002840F0DA8005222021604D02F018FDD9
:10B9A0002B783BB15F4B24215A68002002F010FD38
:10B9B00000232B704FF080520721002002F07CFD05
:10B9C0004FF000620020072102F068FD564BD4F8CA
:10B9D00003201878554B53F82220002840F0B980F6
:10B9E000372102F0F5FC4FF000620121002002F047
:10B9F00063FD55E701F0B2FC4FF00062A078012131
:10BA000002F04CFDA078464A642303FB0023DB7D53
:10BA10007BBB0522202102F0DBFC404DA0782B5C93
:10BA20004BB1404B03EB800324215A6802F0D0FC59
:10BA3000A3780022EA544FF080520721A07802F048
:10BA40003BFD4FF00062A078072102F027FDA078AF
:10BA5000354A60234343D35CD4F803205BB93721D4
:10BA600002F0B6FC4FF000620121A07802F024FD44
:10BA700016E70622CEE72E4B53F820301A44EEE7A5
:10BA800001F06CFC4FF00062A078314602F006FD38
:10BA9000A078234A642303FB0023DB7D73B90522CE
:10BAA000202102F095FC1F4EA07833181B7A012B41
:10BAB00031D005D3022B3DD0002507E00622EFE769
:10BAC000372102F0ABFCD4F803500544A078134FA3
:10BAD0003B5C43B106EB80062421726802F078FCDF
:10BAE000A3780022FA54A0784FF08052072102F088
:10BAF000E3FCA0784FF00062072102F0CFFC2A4659
:10BB0000A078372102F064FC4FF000620121A07898
:10BB100002F0D2FCC4E62121D3E700BF19CDFF1FFC
:10BB200044CDFF1FBCC6FF1FACCDFF1F90CEFF1F33
:10BB300008CDFF1F502102F071FCA278A14B53F8F1
:10BB40002250451BD4F80300BFE706222021002025
:10BB500023E79D4B1B6837211A44002041E700284A
:10BB60007FF4A3AE01F0FAFBA078984A642303FBAC
:10BB70000023DB7D002B33D10522202102F028FC9D
:10BB8000934DA0782B5C4BB1924B03EB80032421A7
:10BB90005A6802F01DFCA3780022EA544FF080524C
:10BBA0000721A07802F088FC4FF000620721A078FE
:10BBB00002F074FCA078884A60234343D15CD4F837
:10BBC0000330864A034452F8232059B9372102F042
:10BBD000FFFB4FF000620121A07802F06DFC5FE6F0
:10BBE0000622CAE7784B53F820301A44EEE7FEF7F6
:10BBF0004BFF55E6FEF728F852E6FEF725F84FE62C
:10BC0000B378022B00F0B880032B00F0BA80002B31
:10BC100040F013817378502B00F0818024D8472B9B
:10BC20006DD011D8422B61D006D8402B43D0412B88
:10BC300058D003232B7044E0452B5AD05CD8442BBA
:10BC4000F7D1674BDB694FE04C2B61D006D8492B0D
:10BC500058D04B2BEDD1624BDB7845E04E2B604B3F
:10BC60005BD058D95B7E3FE0802B67D012D8532B36
:10BC70005BD006D8512B55D0522BDAD1584B1B6ACA
:10BC800032E0552B57D053D3562BD2D1544B93F887
:10BC9000243029E0832B5FD005D8812B52D0822B12
:10BCA000C7D14C4BEBE7852B5BD057D3FF2BC0D1D3
:10BCB0004C4B1B7828E040F2FF70FDF7B8FAC8F84B
:10BCC0000400494B1B78002B3FF4EAAD474B6A68F0
:10BCD0001A60474B002A40F0B2801A6842F008020E
:10BCE0001A60DDE53E4B1B786B60EAE73C4B5B7806
:10BCF000FAE73B4B5B79F7E7394BDB68F4E7384B06
:10BD00009B68F1E7364BDB7D003318BF0123EBE77F
:10BD1000334B9B78E8E75B7DE6E7DB8CE4E7304B71
:10BD20009B7DE1E72E4B1B7DDEE72D4B1B69DBE79F
:10BD30002B4B9B7ED8E72A4BDB7ED5E7254B93F830
:10BD40003430D1E7234B93F83430A3F1040CDCF109
:10BD5000000343EB0C03C7E71E4BCEE7254B1B68E4
:10BD6000C2E71C4A2448136943F2390100FB03135C
:10BD7000136123F00043B7E77278204B53F8223069
:10BD8000B2E77378282B4AD011D8022B45D007D8B8
:10BD9000002B40D0012B7FF44CAF194B5B68A3E71D
:10BDA000092B8ED0272B7FF444AF154BBEE72B2BEE
:10BDB0003BD027D8292B35D02A2B7FF43AAF104B14
:10BDC00040E700BF1CCDFF1F08CDFF1F44CDFF1F64
:10BDD00019CDFF1FBCC6FF1FACCDFF1F90CEFF1FAC
:10BDE0000CC0FF1FF2CEFF1FF3CEFF1FE4CEFF1FDC
:10BDF0008CCEFF1FF4CEFF1F6D4EC64104CFFF1F38
:10BE000010CEFF1F2D2B15D011D32E2B7FF411AF89
:10BE1000964BDB6A68E7954BA1E7944B70E7934B31
:10BE20005B6961E7914B9B695EE7904B27E78F4B1E
:10BE30005B6A59E78D4B9B6A56E70423FAE61A685A
:10BE400022F008021A602BE5B378022B0ED170782D
:10BE5000372808D800F5A7708549800004220144DE
:10BE6000FDF76BF91CE503232B7019E5042388F813
:10BE7000003015E5B378022B0BD170783728F2D853
:10BE800000F5A7707A49800004220144FDF7E8F923
:10BE900006E5042388F8003002E501F0FBFFFFE42B
:10BEA00002F000F8FCE402F005F8724BC8F8040058
:10BEB0001B78002B3FF4F4AC6F4B18606F4B1A6883
:10BEC00018B942F008021A60EAE422F008021A6087
:10BED000E6E4B2782AB1022A0BD0042388F80030B5
:10BEE000DEE47278002A7FF4DBAC1846FCF7AEFE85
:10BEF000D6E47078072806D813B9FCF78DFDCFE497
:10BF0000FCF766FDCCE4FF287FF4CAAC5F1C0ABFD7
:10BF1000594BD8B21878FCF7A3FDC1E4B378012BD4
:10BF200026D02BB1022B27D0042388F800300BE059
:10BF30007078082803D8FCF7A4FD686004E00A289C
:10BF400011D10023C8F804304A4B1B78002B3FF472
:10BF5000A7AC494B6A681A60484B8AB91A6842F024
:10BF600008021A609CE4FF28EED1FCF7F5FDE4E737
:10BF7000707801F0E9FFE0E77078FCF7B7FDDCE7E7
:10BF80001A6822F008021A608AE4106818441060E7
:10BF900012683A4B0ABB1A6842F008021A607FE442
:10BFA0001068C01AF3E710685843F0E7106890FB78
:10BFB000F3F0ECE7116891FBF3F003FB101313604F
:10BFC000E6E710681840E2E710681843DFE71068FA
:10BFD0005840DCE71368DB43F1E71A6822F00802F7
:10BFE0001A605DE4244A1168244A8B4213680ADA15
:10BFF00023F0030343F004031360136869B943F0AB
:10C00000080313604CE40BBF23F0060323F0050381
:10C0100043F0010343F00203EEE723F0080313604B
:10C020003EE472780C2A3FF63BACDFE802F0070FE3
:10C03000172B333C464F58616A737C000F4A1268D5
:10C0400016077FF52DAC0E4A136229E40B4A1268DD
:10C0500015073FF525AC0A4A136221E4074A126826
:10C06000D4077FF51DAC064A136219E410CEFF1FFA
:10C07000CCC9FF1FF3CEFF1FE4CEFF1F8CCEFF1FE6
:10C08000BCC6FF1FA74A1268D0073FF509ACA64AF5
:10C09000136205E4A34A126851077FF501ACA24A76
:10C0A0001362FFF7FDBB9F4A126812F0050F3FF4C1
:10C0B000F7AB9D4A1362FFF7F3BB9A4A12689207E7
:10C0C0007FF5EEAB984A1362FFF7EABB954A126818
:10C0D00097073FF4E5AB944A1362FFF7E1BB914A3F
:10C0E0001268D6067FF5DCAB8F4A1362FFF7D8BB28
:10C0F0008C4A126895067FF5D3AB8B4A1362FFF723
:10C10000CFBB884A126854067FF5CAAB864A1362D1
:10C11000FFF7C6BB834A126810067FF5C1AB824A9F
:10C120001362FFF7BDBB7F4A1268D1057FF5B8AB3C
:10C130007D4A1362FFF7B4BB7B4A1362FFF7B0BBC3
:10C14000794A936B002B3FF4ABAB013B936302EB5B
:10C150008303DB6B1362FFF7A3BB73782E2B04D82A
:10C16000724A0121D154FFF79BBBFF2B7FF47BAEBA
:10C170006D4B012283F85C20FFF792BB73782E2B66
:10C1800004D86A4A0021D154FFF78ABBFF2B7FF401
:10C190006AAE654B002283F85C20FFF781BBFCF799
:10C1A0005BFA6B6EC01A00282B6EB8BF40429842F3
:10C1B00095BF2B6A002303F1FF3385F8243098BF25
:10C1C0002B62FFF76DBBA07801F074FE40B9554AB1
:10C1D00085F82400136823F010031360FFF760BB99
:10C1E0002B6E9BB1FCF738FA6B6EC01A00282B6ED1
:10C1F000B8BF4042984209D94A4A002385F8243002
:10C20000136843F010031360FFF74ABB2B6A013B2E
:10C210002B62FFF745BBA0780F2102F0FFF810F06A
:10C22000010409D03F4A002385F82430136823F025
:10C2300010031360FFF734BB2B6E93B1FCF70CFABD
:10C240006B6EC01A00282B6EB8BF4042984208D9C6
:10C25000344A85F82440136843F010031360FFF755
:10C260001FBB2B6A013B2B62FFF71ABBA0780F2183
:10C2700002F0D4F810F0800409D02A4A002385F88F
:10C280002430136823F010031360FFF709BB2B6EF3
:10C2900093B1FCF7E1F96B6EC01A00282B6EB8BFA2
:10C2A0004042984208D91F4A85F82440136843F059
:10C2B00010031360FFF7F4BA2B6A013B2B62FFF700
:10C2C000EFBAA0780F2102F0A9F810F4807409D019
:10C2D000144A002385F82430136823F010031360F8
:10C2E000FFF7DEBA2B6E93B1FCF7B6F96B6EC01A8E
:10C2F00000282B6EB8BF4042984208D9094A85F8F9
:10C300002440136843F010031360FFF7C9BA2B6A87
:10C31000013B2B62FFF7C4BA034B002283F83420A1
:10C32000FFF7BEBA8CCEFF1FBCC6FF1F52CEFF1F49
:10C33000FF2A7FF4BAAA9C4D70B94FF4C364A4F2EB
:10C3400014612046042229440434FCF7F6FEB4F5B7
:10C35000CD6FF4D1FFF7A4BA00F285108000A0F2EF
:10C36000146104222944FCF7E8FEFFF799BA7078BB
:10C3700014283FF678ADB378CBB98B4B53F8202017
:10C380008A4BC8F804201B78002B3FF489AA884BFD
:10C390001A60884B2AB91A6842F008021A60FFF73F
:10C3A0007FBA1A6822F008021A60FFF779BAFF2BE9
:10C3B0007FF47BAA7C4D70B94FF4C364A4F214617E
:10C3C0002046042229440434FCF74AFFB4F5CD6F1B
:10C3D000F4D1FFF765BA00F285108000A0F2146175
:10C3E00004222944FCF73CFFFFF75ABA7678142E52
:10C3F0003FF639ADA07807061BD5C10706D5212128
:10C40000002002F00BF8684B43F826006A4B9B7E35
:10C41000002B3FF445AA607800283FF441AA00F2BF
:10C4200085106649800004220144FCF786FEFFF770
:10C4300037BA00287FF439AA212101F0EFFF5E4BC3
:10C4400059499B7E41F82600002B3FF429AA6378C6
:10C45000002B3FF425AAA0781C1803F2851318447A
:10C46000042201EB84018000FCF767FEFFF718BA95
:10C4700072784F4B0A2A0CD8DFE802F006151A1F13
:10C48000252D32373C4145004D491A6809680A4458
:10C490001A601A68474B002A3AD11A6842F008021B
:10C4A0001A60FFF7FDB946491A680968521AEFE7A2
:10C4B000434A196812684A43EAE741491A68096819
:10C4C00092FBF1F2E4E73E4A1868116890FBF1F242
:10C4D00001FB1202DCE73A491A6809680A40D7E70B
:10C4E00037491A6809680A43D2E735491A68096862
:10C4F0004A40CDE732490A68D2430A60C9E7196861
:10C500002F4A1160C5E72E4A196810681860F8E7CD
:10C510001A6822F008021A60FFF7C2B9244B1B68A0
:10C52000C6F80330FEF7B0FAFFF7BAB97378052BF7
:10C530003FF6B6A9DFE803F0030A11181F261D4ACB
:10C54000136803F00F031360FFF7AAB9194A1368C1
:10C5500023F010031360FFF7A3B9164A136823F002
:10C5600020031360FFF79CB9124A136823F04003BD
:10C570001360FFF795B90F4A136823F08003136027
:10C58000FFF78EB90B4A136823F480731360FFF72B
:10C5900087B971782E293FF666AC0A4A02EB810210
:10C5A0009366FFF77DB900BF90CEFF1FF3CEFF1F4C
:10C5B000E4CEFF1F8CCEFF1F0CC0FF1F7CC8FF1FE7
:10C5C00000CFFF1FBCC6FF1FC74BC84AD3F82411BA
:10C5D0001160C74AD3F828111160D3F82C211A62D0
:10C5E000C44AD3F830111160D3F8342183F82420E1
:10C5F000D3F838215A66D3F83C211A6693F84011D3
:10C60000BD4A505C08B101205054002283F84421F7
:10C61000FFF746B900F01CFEFFF742B900F019FE23
:10C62000FFF73EB900F016FEFFF73AB900F014FE2E
:10C63000FFF736B900F011FEFFF732B900F00EFE39
:10C64000FFF72EB9A84B002283F83420FFF728B952
:10C65000727832B1012A0AD0032388F80030FFF73C
:10C660001FB9A14B012283F83420FFF719B940F21A
:10C67000FE718B423FF619A99B4981F834200B6269
:10C68000FFF70EB9984A9C48002382F85C3082F884
:10C69000443102F168044FF0FF35194644F8235045
:10C6A000C15401332F2BF9D1904B82F8341019600B
:10C6B0008F4B116219608F4B916382F824101960BF
:10C6C000FFF7EEB8127D92070CD440F2FE7293424F
:10C6D0003FF6EBA8844A042182F83410C2F84831AE
:10C6E000FFF7DEB8082388F80030FFF7D9B87E4B93
:10C6F000002283F83420FFF7D3B82B460022E254FF
:10C700000133082BFBD123782372FFF7C9B8737864
:10C71000012B1AD006D3022B24D0032388F8003033
:10C72000FFF7BEB8754B01221A70754B754A9B789E
:10C730001370754B196800230139013311F8010F8B
:10C74000D054082BF9D1FFF7ABB8042288F80720A2
:10C7500088F805305722082388F8062088F8043026
:10C76000FFF79EB8654B694801221A70644B654A11
:10C770009B781370002301331918082B11F8091C3A
:10C78000D154F8D1FFF78CB87378032B3FF688A803
:10C79000DFE803F00214252B534B93F8342088F87C
:10C7A000072093F82420D3F8483188F806201A0A85
:10C7B00088F8052088F80430FFF772B84A4B93F8E0
:10C7C000342088F8072093F824201B6A88F8062074
:10C7D0001A0A88F8052088F80430FFF761B8434B3F
:10C7E0001B68C8F80430FFF75BB8414B1B68C8F8FA
:10C7F0000430FFF755B87278002A7FF451A8B17859
:10C8000000297FF44DA840F2D24293427FF448A819
:10C8100040F2FF70FCF732FCFCF797FB0120FBF7BE
:10C82000F7FFFFF73DB80122FEF7BEBF747834B1C1
:10C83000012C16D0032388F80030FFF731B804220A
:10C84000694640F2FB70FCF70BFD009BD6F8032015
:10C850009A4206BF0123C8F80430C8F80440FFF725
:10C860001FB8B3782A2B07D10422294940F2FB7064
:10C87000FCF763FCFFF714B8032388F80030FFF7D8
:10C880000FB8194CD4F85001002104F5AA72814266
:10C890003FF406A852F821509D4201F1010521D133
:10C8A00002EB8503043B0138814215D3C4F85001E3
:10C8B000FEF7F6BF0C4AD2F8501109299DBF481C5B
:10C8C000C2F8500102EB8102092394BFC2F854312F
:10C8D00088F80030FEF7E4BF53F8042F43F8042C27
:10C8E0000131E1E72946D2E7BCC6FF1FE4CEFF1FB6
:10C8F00000CFFF1F8CCEFF1F52CEFF1FE8CEFF1FC1
:10C900000CC0FF1FE9CEFF1F08C0FF1F0080000002
:10C9100087CEFF1F334A0023C2F85031194602F573
:10C92000AA7242F8231001330A2BFAD1FEF7B8BFDE
:10C930000A23C8F80430FEF7B3BF032388F8003099
:10C94000FEF7AEBF7378812B7EF4AFAFB378922B36
:10C950007EF4ABAFB379A32B7EF4A7AF7379B42B7E
:10C960007EF4A3AF3379C52B7EF49FAFF378D62B3B
:10C970007EF49BAFFCF713FAFBF76EFE0446FBF761
:10C980006BFE001B0028B8BF4042B0F57A7FF6DB93
:10C99000FBF73CFF144B00221A604FF0FF32C3F844
:10C9A0007021C3F87022C3F87421C3F87422C3F84D
:10C9B0007821C3F87822C3F87C21C3F87C220B4B82
:10C9C0000B4A1A600120FBF723FFFEF769BF40F214
:10C9D000D24293427EF464AF024B012283F87C2161
:10C9E000FEF75EBFBCC6FF1F10E000E000C0FF1FE7
:10C9F00078563412F7B50F4C07460E4694E80300FC
:10CA00008DE803000C49C1F803300C4B8A700022FA
:10CA10000F704E701A70FEF755FD094A217882F8A2
:10CA200035109DE80300636884E80300184603B0EE
:10CA3000F0BD00BFF8CEFF1F84CEFF1FF3CEFF1F57
:10CA4000BCC6FF1FF7B504461F4A63781370A3786E
:10CA50005370E37893702379937163795371A37959
:10CA60001A4D1371E379D3700E4695E80300184B05
:10CA700000221A708DE80300FEF724FD154B1A788A
:10CA80006F462B469AB9327072702A78B2706A7803
:10CA9000F270EA793271AA7972716A79B2712A797F
:10CAA000F27197E8030083E8030003B0F0BD012AA8
:10CAB000F7D10948721EF11D10F8014F02F8014F1D
:10CAC0008A42F9D1EDE700BF84CEFF1FF8CEFF1FE9
:10CAD000F3CEFF1FE8CEFF1FE9CEFF1F2DE9F04385
:10CAE000994B9A4C1B788FB06BB1994B1B78063BD6
:10CAF000DBB2192B04D8974A22FA03F3D90702D4E0
:10CB0000002384F84C3194F84C31934E5A1E012A7C
:10CB100051D89249012BCA68079214BF08230723F2
:10CB20008DF81830327894F87D318DF81930002363
:10CB30008DF81A30002A33D18B688DF82030884B5D
:10CB40008DF8272019788DF8211059788DF822104A
:10CB5000D9798DF8231099798DF8241059791B799A
:10CB60008DF825108DF8263006A801F00DFB002861
:10CB700000F01E837B4B1A789846002A00F01E8135
:10CB8000794B7A4F1B78013B062B00F21381DFE8CB
:10CB900013F0F100F10058011101110111017F01A1
:10CBA000012AE1D17248013306AA1A44195CD171F5
:10CBB000082BF8D1D8E7032B3DD1337883BBDFF8BE
:10CBC0009C81674F98F8020098F801503B78054423
:10CBD0001D447B781D44FB791D44BB791D447B7942
:10CBE0001D443B791D44FBF771FD98F80100FBF7EC
:10CBF0006DFD3878FBF76AFD7878FBF767FDF8790B
:10CC0000FBF764FDB879FBF761FD7879FBF75EFD12
:10CC10003879EDB2FBF75AFD2846FBF757FDA9E737
:10CC2000012BA7D1524F0025785D0135FBF74EFD52
:10CC3000092DF9D19EE7042B2BD1484FDFF8208135
:10CC4000B8787D78002301220544154488F8013026
:10CC500088F80020C8F80430FBF738FD7878FBF737
:10CC600035FD98F80000FBF731FD98F80100FBF75F
:10CC70002DFD98F80700FBF729FD98F80600FBF753
:10CC800025FD98F80500FBF721FDEDB298F80400AA
:10CC9000C0E7072B37D1337853BB304B9F7893F8DD
:10CCA00001802F4B8DF800701D785878D9798DF858
:10CCB000025047443D449A798DF80300284493F884
:10CCC00005C08DF80410014493F804E08DF80520A8
:10CCD0000A440CEB020373448DF801808DF806C002
:10CCE0008DF807E08DF808306846FCF755F841E705
:10CCF000012BF9D11E4900235A5C0DF803200133A2
:10CD0000092BF9D1F0E7082B7FF434AF144A13490B
:10CD1000002301205370107053608A7849788DF891
:10CD200000200A4402448DF801108DF802008DF8AD
:10CD300003308DF804308DF805308DF806308DF80D
:10CD400007308DF80820CFE7F2CEFF1FBCC6FF1FCB
:10CD500084CEFF1F11020002E8CEFF1F0CC0FF1F90
:10CD6000F8CEFF1F81CEFF1F4ECEFF1F1ACDFF1F33
:10CD7000E9CEFF1FAD4A397893688DF830308023B3
:10CD80008DF831308A238DF8323000238DF833301E
:10CD90008DF834308DF835308DF836108DF8293017
:10CDA00007218DF82A300AA8D3688DF828100B9334
:10CDB00001F0EAF900233B7088F80030002384F882
:10CDC0004C31337094F87C3113B10120FBF720FD16
:10CDD00006A801F065F90646002800F03F81944B53
:10CDE0009DF820201A709DF821205A709DF822206D
:10CDF0009A709DF823209A719DF824205A719DF80D
:10CE000025201A719DF82620DA709DF8193084F8D3
:10CE10007D31FBF721FC874B1860874B00221A708D
:10CE20009DF81830072B0CBF0123022384F84C31E6
:10CE300094F834305A1E012A4AD9052B48D00122D1
:10CE400047E0DFF8E8913B7899F8020099F8015043
:10CE500005440A351D44FBF739FC99F80100FBF73E
:10CE600035FC8020FBF732FC8A20FBF72FFC0020EA
:10CE7000FBF72CFC0020FBF729FC0020FBF726FC2D
:10CE8000EDB23878FBF722FC2846FBF71FFC91E750
:10CE9000664A507893788DF80C303A788DF80D000A
:10CEA000802103448DF80E100A338A218DF80F106B
:10CEB0001344002103A88DF810108DF811108DF87F
:10CEC00012108DF813208DF81430FBF765FF71E711
:10CED00000225A4B1A7094F83430042B04D1544B6E
:10CEE00019780A0640F1678194F84C21082A04D881
:10CEF00040F25113D340DF0701D4FEF7E3FA94F870
:10CF00004C31092B6DD1FBF7A7FB63694C4DC01A5F
:10CF100000282A68B8BF4042904208D9494B1A7885
:10CF2000012A04BF02221A70FBF796FB6061FBF72F
:10CF300093FBA3696A68C01A0028B8BF40429042B8
:10CF400008D9404B5A78012A04BF02225A70FBF7D5
:10CF500083FBA061FBF780FBE369AA68C01A002885
:10CF6000B8BF4042904208D9364B9A78012A04BF94
:10CF700002229A70FBF770FBE06194F85C3083B397
:10CF800094F844316BBB2F4A2F481D46D15C0229CF
:10CF900040F0058150F823104E1C00F0FF802B4A12
:10CFA00084F840311268C4F82421294A1268C4F870
:10CFB0002821226AC4F82C21264A21621268C4F86A
:10CFC000302194F82420C4F834210023626EC4F880
:10CFD000382184F82430226EC4F83C21012384F8DF
:10CFE000443194F84C31092B06D194F83420022AAC
:10CFF00004BF052284F83420D4F85021002A00F020
:10D00000D780092B40F0D48094F83430012B40F0C5
:10D01000CF80216A1048002350F823508D4240F001
:10D02000C380052384F83430C2E000BF0CC0FF1F6A
:10D0300084CEFF1F40CEFF1FF8CCFF1FF3CEFF1F93
:10D0400010CEFF1F52CEFF1F24C7FF1FE4CEFF1FCD
:10D0500000CFFF1F8CCEFF1F10C8FF1F03A8FBF7D8
:10D060004DFB054600284ED0FBF760FB08B184F865
:10D070007E6194F87E219DF80C10531CDBB2224493
:10D08000092B84F87E3182F87F117FF424AF5F4A48
:10D0900094F87F1152780023914284F87E317FF416
:10D0A0001AAF5B495A5C01331644082BF6B2F9D12A
:10D0B00094F88731B34222D1564B94F880211A70EC
:10D0C00094F881215A7094F882219A7094F88321FF
:10D0D0009A7194F884215A7194F885211A7194F800
:10D0E0008621DA70FBF7B8FA4B4B4C4A18600023E4
:10D0F0001370032284F84C2184F87E3198E60423CF
:10D1000084F84C31E7E60AAE3046FBF732FE48B30E
:10D110002B46F25C01331544082BEDB2F9D19DF892
:10D120003020AA42ECD13B4B9DF829201A709DF883
:10D130002A205A709DF82B209A709DF82C209A7105
:10D140009DF82D205A719DF82E201A719DF82F20E0
:10D15000DA70FBF781FA304B1860304B00221A70FE
:10D16000072363E694F83430013B012B3FF6B3AE5E
:10D17000226A40F2FE739A420CD8FBF7D5FD48B103
:10D18000206A2449431C2362FBF79EFE092384F88E
:10D190004C3154E6002384F834309CE6D5540133F6
:10D1A0002F2B7FF4F3AE1CE701339A427FF434AFA8
:10D1B0000FB0BDE8F08394F84C01082804D840F281
:10D1C0005112C240D207F3D4154DD3F80330D4F82E
:10D1D00048016B6040F2FE739842697012D80D49A5
:10D1E000FBF782FF0B49D4F84801FBF7EFFE38B19B
:10D1F000D4F848310133C4F8483165232B70D7E7A0
:10D200000723FBE707232B7000230BE70CC0FF1F4E
:10D210003BC8FF1F84CEFF1F48CEFF1F4DCEFF1F10
:10D22000F8CEFF1F704710B5074CFBF715FA2368BF
:10D23000C01AB0F5FA7F05D9044B2022DA60FBF75B
:10D240000BFA206010BD00BF04D3FF1F00F00F4099
:10D250007047704770477047704770477047704716
:10D26000024B185C431F58425841704744C8FF1F87
:10D2700038B505460C46A1B901F0D0F8214620F496
:10D28000E072284601F0A4F860236B431B4AD35C8C
:10D290009BB328464FF000620721BDE8384001F0FB
:10D2A000FDB8002101F0BAF804F00303022B20F4CA
:10D2B000E0721CD0032B1DD0012B01D142F04002A3
:10D2C000630748BF42F4807214F0080418BF42F4A8
:10D2D00000720021284601F07BF8002CD9D12846A5
:10D2E0004FF000620721BDE8384001F0E5B842F098
:10D2F0008002E5E742F0C002E2E738BDACCDFF1F97
:10D3000073B5144C231806465B780D4623B94FF0CD
:10D31000C052072101F0D0F80F4A602303FB062317
:10D3200001229B7D019285EAE572A2EBE572D2B201
:10D33000009206210022304601F020F8002D04EB77
:10D34000060304EB8604B4BF012202225A70656012
:10D3500002B070BD44C8FF1FACCDFF1F184B1A1898
:10D3600073B55178044641B303EB80030025557033
:10D3700007214FF080525D6001F090F84FF000629D
:10D380000721204601F098F860230E4A6343D6181F
:10D39000D35C93B15021204601F040F82121024690
:10D3A000204601F015F8327DB37D0192727D009226
:10D3B00006212A46204600F0E1FF02B070BD00BF02
:10D3C00044C8FF1FACCDFF1F2DE9F347A64D2C7AB3
:10D3D00005F109084CB9E0B2FBF753FB08F804006B
:10D3E0000134082CF7D101232B72DFF8B0A29F4F34
:10D3F000272400264FF00209F0B2FBF742FB18F891
:10D400000630834216D0331D08F806005AF8233040
:10D41000022B0AD0032B02D0012B0BD150B13B5D64
:10D42000012B08BF07F8049004E018B93A5D012AFF
:10D4300000D13B550136082E04F10104DCD18C4C9F
:10D44000E36993B18B4E37787FB9FBF705F98A4BC7
:10D450001B68C01A0028E369B8BF4042984204D94B
:10D46000384601F071F801233370236A93B1834E7B
:10D4700037787FB9FBF7F0F8814B1B68C01A00289A
:10D48000236AB8BF4042984204D9384601F05CF89C
:10D49000012333702221687C7A4E00F0BFFF07021F
:10D4A000687C01F038F80446687C642303FB006361
:10D4B0001B69002B00F0A080002B87EAE772A2EB2B
:10D4C000E772B8BF5B429A4240F396802B189B7C70
:10D4D00043B94FF08062012100F0E0FF6B7C012234
:10D4E0002B449A7404F00903092B31D1687C5F49FD
:10D4F000C21C8B5CDBB2012B0ABF4FF0020E8B5CAF
:10D5000001F802E060490A7818BFB3FA83F342FADF
:10D5100000FE18BF5B091EF0010F15D04FF0010C83
:10D52000DFF87C810CFA00FE88F800E0DFF87481F7
:10D5300088F800C0DFF870C19CF800C0BCF1000F93
:10D5400002D122EA0E020A7013B1092100F0F0FFA5
:10D55000A2000CD5687C454A00F10F03D15C01297B
:10D5600004BF0221D1544FF0005100F0E1FF230528
:10D5700005D527B94FF40061687C00F0D9FFE004BD
:10D5800005D527B94FF48051687C00F0D1FFA10484
:10D5900005D527B94FF40051687C00F0C9FF62043B
:10D5A00005D527B94FF48041687C00F0C1FFFBF737
:10D5B00053F86B69C01A0028B8BF40420A284FDDF3
:10D5C000687C324B324F03440193324B0344009347
:10D5D000314B002203EB80031146FCF7C5FA6C7C4B
:10D5E0002A5D6023052A26D8DFE812F014006000C7
:10D5F000A800EF00010144012B189B7C002B3FF495
:10D6000071AF4FF08062012100F056FF6B7C002269
:10D610002B4466E76343FB5C6BB1204600F04AFC99
:10D6200048B9642303FB04662046717AC908FCF7F5
:10D630007BF901232B55687C00F0ACF96C7C6023EE
:10D640006343FB5C3BB12B195B78012B00F05881E5
:10D65000022B00F0618100236B74FAF7FDFF686113
:10D6600002B0BDE8F08700BF44C8FF1F52CEFF1FC5
:10D670000CC0FF1F4DCEFF1F48CEFF1FF8CCFF1F71
:10D6800040CEFF1F44CDFF1F20CDFF1F41CDFF1F08
:10D69000ACCDFF1F0CCDFF1F24CDFF1F10CEFF1FF1
:10D6A0001ACDFF1F81CEFF1F00CDFF1F00220521D5
:10D6B000204600F08DFE602202FB04722046117DA0
:10D6C000937D0191527D00920621002200F056FECA
:10D6D0007921204600F0A2FE7F281BDCC0F18006E5
:10D6E00004222021204600F073FE8F4A2421204688
:10D6F00000F06EFE2121204600F090FE37218219B5
:10D70000204600F065FEFAF7A7FF05EB8403986159
:10D7100002238FE7B0F5C07F02DAC0F5C076DFE7FD
:10D72000B0F5207F02DAC0F52076D9E7B0F5607F4A
:10D73000B4BFC0F56076C0F59066D1E7FAF78CFF0C
:10D7400005EB84039B69C01A0028B8BF4042B0F5BE
:10D750007A7F7FF770AF642303FB0466F66956B1E6
:10D760002121204600F05AFE50210246204600F0BA
:10D770002FFE03235EE732462021204600F028FEDC
:10D7800032462421204600F023FE5021204600F09E
:10D7900045FE21210246204600F01AFE21212046A6
:10D7A00000F03CFE37210246204600F011FE042224
:10D7B0002021204600F00CFE5B4A2421204600F088
:10D7C00007FE5A4B01221A55D3E74FF0C0520721EA
:10D7D000204600F071FE564A0721204600F05EFE0A
:10D7E000FAF73AFF05EB84039861042322E7FAF77E
:10D7F00033FF05EB84039B69C01A0028B8BF404281
:10D80000B0F57A7F7FF717AF4FF019420721204616
:10D8100000F052FE642303FB0466737E0BB11B070A
:10D8200025D54FF020620721204600F037FE8022E8
:10D830000521204600F0CCFD5921204600F0EEFDE8
:10D84000602303FB0473002218613A4B50212046E9
:10D8500043F8242000F0E2FD21210646204600F096
:10D86000DDFD354B301A43F824000523E2E64FF086
:10D870000072D8E7634317F80380B8F1000F7FF414
:10D88000DAAE2046FFF76AFD4FF00462072120461A
:10D8900000F012FE03220521204600F099FD6423CA
:10D8A00003FB04660621B37DB27A0193737A009379
:10D8B0002046434600F062FD1F212046FCF734F865
:10D8C000F37D05F80480CBB901222021204600F029
:10D8D0007FFD00222421204600F07AFD21212046F0
:10D8E00000F09CFD134B53F824202121821A20467E
:10D8F00000F06EFD0D4B01221A559CE60222E4E772
:10D900005021204600F08AFDA0F5C332A03A212123
:10D91000204600F05DFD9EE65021204600F07EFD91
:10D9200000F5C332A032F2E740420F0019CDFF1FCD
:10D930000000408108CDFF1F1CCDFF1F024B03EBF1
:10D9400080004068704700BF44C8FF1F38B5104AC8
:10D95000642303FB00230446DB7D0D46B3B901229B
:10D96000202100F035FD20464FF08052072100F0C5
:10D9700095FD20464FF00062072100F09DFD2A46EC
:10D9800020462421BDE8384000F022BD0222E7E70E
:10D9900044CDFF1F2DE9F84F0F21C14D044600F083
:10D9A0003DFD64236343E9184FEA102B0A7A4F6860
:10D9B00012F0400F14BFEB5855F803904FEAD01007
:10D9C00016BF0BF0010A00F0010A00F0010BA84697
:10D9D0001ABFC3F100097F420BF0010B150602F0DC
:10D9E0003F06204612D500F08BFEB0FA80F04009C9
:10D9F000731E072B00F2AC81DFE813F00E000E005F
:10DA00000E000E003B013B013B013B0100F078FEA4
:10DA1000003018BF0120EBE7A24D2B5D013B0E2B20
:10DA200000F29681DFE813F00F001E002D003A008F
:10DA30004A00540063007100B200D900DF00940175
:10DA40001D01270222020121204600F0E7FC05EB20
:10DA5000840301225860023E934B96421A551BD80C
:10DA6000022333E005EB84035A6842F002020121ED
:10DA7000204600F0ADFC49462046FFF767FF032330
:10DA800024E0BBF1000F00F063812121204600F06B
:10DA9000C5FC864B43F82400042317E005EB840300
:10DAA0005A6842F001020121204600F091FCC9F1C0
:10DAB00000012046FFF74AFF052307E0BAF1000FF7
:10DAC00000F04681204600F03FFD06232B553FE144
:10DAD00005EB840301215A68204622F0030200F07E
:10DAE00077FC39462046FFF731FF0723EEE7BAF10E
:10DAF000000F40F02D8151462046FFF727FF794265
:10DB00002046FFF723FF0823E0E7BAF1000F00F0FB
:10DB10001F812121204600F081FC0021064620467D
:10DB2000FFF714FF614A52F824309B1B42F824305F
:10DB300005EB840301215A68204622F0030200F01D
:10DB400047FC642303FB048898F81730E3B90522E7
:10DB50002021204600F03CFC3A462421204600F0DB
:10DB600037FC4FF080520721204600F0A5FC4FF013
:10DB700000620721204600F091FC32463721204602
:10DB800000F026FC0923A1E70622E1E70F21204649
:10DB900000F044FCC10740F1DB802121204600F069
:10DBA0003DFC434B002118602046FFF7CFFE0022CA
:10DBB0003721204600F00CFC00222121204600F0F5
:10DBC00007FC5021204600F029FC033E394B012E72
:10DBD00043F824004BD87942CDE0BAF1000F00F0B1
:10DBE000B7800B2372E7BAF1000F40F0B18021211A
:10DBF000204600F013FC514606462046FFF7A6FEDD
:10DC0000022396FBF3F605EB840301215A682046B4
:10DC100022F0030200F0DCFB642303FB048898F885
:10DC20001730E3B905222021204600F0D1FB3A4607
:10DC30002421204600F0CCFB4FF0805207212046E3
:10DC400000F03AFC4FF000620721204600F026FC6D
:10DC500032463721204600F0BBFB0D2336E7062273
:10DC6000E1E70F21204600F0D9FBC20770D50E2353
:10DC70002CE70C4D2B5D013B0E2B69D8DFE813F030
:10DC80001C002C003D004B005C0068006A0068002E
:10DC9000680092009C008000D100FB00F60000BFED
:10DCA00044CDFF1F60C8FF1F19CDFF1FFCCCFF1F15
:10DCB0000CCEFF1F1CCDFF1F734B012120461955B1
:10DCC00000F0ACFB05EB8403062E58603FF4C8AEB1
:10DCD000082E7FF4E1AEC3E6062E05D105EB8403E2
:10DCE0005A6822F00302C0E6082E7FF4C4AE05EBAA
:10DCF00084035A6822F00302B9E6731F012B07D888
:10DD0000BBF1000F04D0062E3FF4C6AE0F23DDE6B4
:10DD1000F0B10C23DAE6052E05D105EB84035A6831
:10DD200022F00302BDE6072E7FF4C1AE05EB8403AB
:10DD30005A6822F00302B6E6731F012B05D8BAF128
:10DD4000000F02D0052EE1D18AE600287FF4CDAE87
:10DD5000BDE8F88F0028FBD1073E012E0AD905EB5C
:10DD6000840301215A6822F0030242F00202204695
:10DD700000F02EFB39462046FFF7E8FD0A23A5E612
:10DD80000028E5D1073E012E7FF625AF05EB840381
:10DD900001215A6822F0030242F00102204600F0FD
:10DDA00017FB18E70028D3D02121204600F036FBCE
:10DDB00005EB8403986014E70028C9D1212120468F
:10DDC000A60000F02BFBAB1981465A68012122F016
:10DDD0000302204600F0FCFA642303FB048898F851
:10DDE0001730E3B905222021204600F0F1FA3A4627
:10DDF0002421204600F0ECFA2E444FF080520721F7
:10DE0000204600F059FB4FF000620721204600F049
:10DE100045FBB2689144022299FBF2F219E706220F
:10DE2000E1E70F21204600F0F9FAC30790D50E2351
:10DE3000212120462B5500F0F1FA144B00211860E7
:10DE40002046FFF783FD00223721204600F0C0FA6C
:10DE500000222121204600F0BBFA5021204600F08C
:10DE6000DDFA0B4B43F82400BDE8F88F0021204673
:10DE7000FFF76CFDFBE605EB840301215A682046A1
:10DE800000F0A6FA002321E619CDFF1F0CCEFF1FDC
:10DE90001CCDFF1F024B1A5C0AB901221A547047AD
:10DEA00060C8FF1F024B1A5C0AB10F221A54704758
:10DEB00060C8FF1F014B185C704700BF60C8FF1FA0
:10DEC0000E4B1A6802F01F02052A0AD0062A0ED04D
:10DED000042A10D11A690A4992B20A8045221A60AE
:10DEE00070471A69064992B28A804622F7E71A6992
:10DEF000034992B24A804422F1E700BF00B00B40D0
:10DF00006CC8FF1F0E4B41F230013A205A5842F0C4
:10DF100000625A5041F23C015A5842F000625A5095
:10DF200003F5E8230C229A6006491022DA600022E9
:10DF30005A620A624A628A6244221A6000F008BC8D
:10DF40000070044000B0044009282BD8DFE800F03E
:10DF5000050A0D1014172A2A1A25134B1888C0F326
:10DF60000B107047104B5888F9E70F4B9888F6E76D
:10DF70000D4B188880B270470B4B5888FAE70A4B54
:10DF80009888F7E7084B588883B24FF49870584345
:10DF90004FF6FF7390FBF3F07047034B988883B202
:10DFA0003420F4E7002070476CC8FF1F30B52E4DB9
:10DFB00041F23C042B5943F010032B512B4B4FF4EF
:10DFC00000749C646FF4F875DC64A3F51833A4F155
:10DFD0003E542C441C604FF400545C60244C1C6084
:10DFE0001C68E401FCD50138072834D8DFE800F0CC
:10DFF000312F2D2B293327041E4858601E4B00203B
:10E0000058631E4818601E484FF0806400EA81453E
:10E01000C3F88040C3F88450FAB100EA8240C3F8E4
:10E020009040C3F894004FF08460C3F8A000C3F898
:10E03000A410AAB1C3F8B000C3F8B42030BD114891
:10E04000DBE71148D9E71148D7E71148D5E7114870
:10E05000D3E71148D1E71148CFE7C3F89020E2E7B2
:10E06000C3F8B02030BD00BF0070044000A00440E1
:10E070000F0080508320FC01004002400F00800010
:10E080000000FC1F8720FE028720FE0B8720FE0E6B
:10E090008720FE1D8720FE4A8720FE958720FE05EB
:10E0A000384AD2F88030C3F30363022B5FD0D2F832
:10E0B0009030C3F30363022B5BD0D2F8A030C3F3DC
:10E0C0000363022B06D0D2F8B030C3F30363022BF4
:10E0D00056D103231B0103F1402202F50032D2F88E
:10E0E0008010C1F303410170D2F8801011F4801147
:10E0F00018BF01218170D2F8801011F4001118BFEF
:10E10000012141704178B1BBD2F88410C1F38A413A
:10E1100003F1402303F500334160D3F88810090E62
:10E120000172D3F88810090C4172D3F88810090ADB
:10E130008172D3F88810C172D3F88C10090E017364
:10E14000D3F88C10090C4173D3F88C10090A817331
:10E15000D3F88C30C373D2F880309B024CBF4FF0A1
:10E1600084634FF08063C2F8803001207047002341
:10E17000B0E70123AEE7D2F8841021F06041C7E791
:10E180000020704700400240184AD2F87031C3F3B3
:10E1900003630C2B10B527D04478436804B3C3F352
:10E1A0001103C2F874318368104A1BBAC2F878317F
:10E1B000C3681BBAC2F87C318378002C14BF4FF0BF
:10E1C00042624FF040620BB142F4801203781B04AC
:10E1D00003F470231343054A0120C2F8703110BDC7
:10E1E000034901EA8343DCE7002010BD0040024000
:10E1F0000000FC1F0B4B4FF00062C3F870214FF47E
:10E200008022C3F87421084AC3F878216FF484711E
:10E21000A2F166320A44C3F87C21044AC3F8702193
:10E22000704700BF00400240785634120000080CCE
:10E2300013B5164C0C23A28F00930A21042300204F
:10E2400000F048F9002108464FF4805200F0C0F871
:10E25000E2695421002000F0BBF800221046502152
:10E2600000F0B6F80A4B5A6CFF20082183F84000F2
:10E2700083F8411001900091D3B26321C2F30722C9
:10E28000002000F07BF802B010BD00BF44CDFF1F9E
:10E29000ACCDFF1F38B50D460721044600F0BEF88F
:10E2A000EB074CBF40F0800220F08002A8074CBF73
:10E2B00042F4807222F4807269074CBF42F010026F
:10E2C00022F010022B074CBF42F4007222F40072BD
:10E2D000E8064CBF42F0040222F00402A9064CBF3B
:10E2E00042F0080222F008026B064CBF42F0200206
:10E2F00022F0200228064CBF42F0400222F04002E9
:10E30000E9054CBF42F0020222F00202AB052046B2
:10E310004CBF42F4806222F480620721BDE838409D
:10E3200000F056B8072108B500F078F8C0F3C01324
:10E33000C20548BF43F00203C10648BF43F00403CF
:10E34000820548BF43F00803410748BF43F010036C
:10E35000020748BF43F02003810648BF43F0400353
:10E36000420648BF43F08003810748BF43F48073EF
:10E37000420548BF43F40073184608BD2DE9F0413B
:10E380001F46124B9DF8186033F810409DF81C5042
:10E39000904641F0800100222046FAF751FD4146A7
:10E3A00000222046FAF74CFD394600222046FAF7B3
:10E3B00047FD314600222046FAF742FD2946204615
:10E3C0000122BDE8F041FAF73BBD00BF4CC0FF1F82
:10E3D00038B5114B33F81040154641F0800100224A
:10E3E0002046FAF72DFD290E00222046FAF728FDD7
:10E3F000C5F3074100222046FAF722FDC5F30721A5
:10E4000000222046FAF71CFDE9B220460122BDE8B1
:10E410003840FAF715BD00BF4CC0FF1F38B51E4B82
:10E4200033F81040002220460D46FAF709FD00227D
:10E4300011462046FAF704FD002211462046FAF75D
:10E44000FFFC002211462046FAF7FAFC01220021C7
:10E450002046FAF7F5FC294600222046FAF7F0FCA0
:10E46000002211462046FAF7EBFC00221146050275
:10E470002046FAF7E5FC0022114605432046FAF74C
:10E48000DFFC2D020543012200212046FAF7D8FCCB
:10E490002D02284338BD00BF4CC0FF1F70B5044695
:10E4A0000D461646FFF7BAFF294640EA0602204607
:10E4B000BDE87040FFF78CBF70B504460D461646A8
:10E4C000FFF7ACFF294620EA06022046BDE870406F
:10E4D000FFF77EBF2DE9F8439DF8209098460F4640
:10E4E000064614460025FFF799FFC1444146012323
:10E4F00049450BD304FA08F444402C4080EA040256
:10E5000039463046BDE8F843FFF762BF03FA01F22F
:10E5100015430131ECE710B50C2104464FF0FF32F2
:10E52000FFF756FF20460E21BDE81040FFF776BFEB
:10E5300010B5CA4304460C21FFF74AFF20460E21BE
:10E54000BDE81040FFF76ABF10B5084BC4B2012206
:10E550001A54202120460022FFF73AFF20460022CD
:10E560002421BDE81040FFF733BF00BF19CDFF1FC6
:10E5700013B5002108464FF48052FFF729FF8A2285
:10E5800004210020FFF724FF032205210020FFF7CC
:10E590001FFF042220210020FFF71AFF002210464F
:10E5A0003721FFF715FF002210462121FFF710FF4A
:10E5B0004FF4480224210020FFF70AFF484C4FF493
:10E5C000483228210020FFF703FF4FF44832292169
:10E5D0000020FFF7FDFEA37DA27A0193637A0093EA
:10E5E000002318460621FFF7C9FEA38A3D4A3E4C88
:10E5F0005A4315210020FFF7EBFE626860210020DE
:10E60000FFF7E6FEA26861210020FFF7E1FEE38943
:10E61000227B1C2143EA02420020FFF7D9FE226937
:10E6200059210020FFF7D4FE226A5A210020FFF76B
:10E63000CFFE626A5B210020FFF7CAFEA26A94F84F
:10E640002C30D1B2C2F30722009200220191104671
:10E650005D21FFF793FE226B5E210020FFF7B8FEDD
:10E66000A26918210020FFF7B3FEE26919210020FA
:10E67000FFF7AEFE626B5C210020FFF7A9FEA26BE4
:10E680005F210020FFF7A4FEE26B52210020FFF77C
:10E690009FFE94F84030626C019394F841300093EF
:10E6A0006321D3B20020C2F30722FFF767FE94F87C
:10E6B0004830002422462046019400947D21FFF733
:10E6C0005DFE20464FF440320121FFF781FE6FF0DE
:10E6D00000423521204602B0BDE81040FFF778BE69
:10E6E00044CDFF1F00710200ACCDFF1F034B102271
:10E6F0009A6000BF00BF00BF5A607047C0F00F4073
:10E7000008B50F21FFF78AFEC0F3003008BD0002F4
:10E710007047800070470012704780107047704744
:10E72000FEE74FF0E023084AC3F8082D074A4CF2F1
:10E730002053D3814DF62813D381138823F001038E
:10E740001B041B0C13807047008000000020054054
:10E75000802800F01F014FF001030F4A04DD8B40B9
:10E76000C2F88C31D3607047402804DD8B40C2F87A
:10E77000883193607047202804DD8B40C2F88431D3
:10E7800053607047404200F01F0058BF41428B4029
:10E79000C2F880311360704700E100E0802800F08B
:10E7A0001F024FF001030D4903DD9340C1F88C3087
:10E7B0007047402803DD9340C1F888307047202817
:10E7C00003DD9340C1F884307047404200F01F00E1
:10E7D00058BF42429340C1F88030704700E100E0EA
:10E7E000074B1A78D2B2012A02D1222903D15A70DA
:10E7F00001225A7070472129FAD10022F7E700BFA1
:10E8000080C8FF1F70B5154611B91B4B197070BD3C
:10E81000022903D1184B01221A7070BD04291AD1A4
:10E82000154B5B78012B25D19488402C28BF4024C0
:10E8300000235E1CDBB2A34207D300231A46022149
:10E840001846BDE8704000F047BF2A68D05C00F071
:10E85000C3F83346EDE7032906D1074A5378012B65
:10E8600008D100239370E9E7052901BF024B00227C
:10E870001A705A7070BD00BF80C8FF1F10B50446E3
:10E88000204600F0C1F80028FAD110BD704738B515
:10E890000A4C012502460B4600202946A57000F0CF
:10E8A000F5FA224618B10023A370122038BD9378E0
:10E8B00003F0FF00002BFAD138BD00BF80C8FF1F56
:10E8C000F8B506460F4600F0F4FC0E4B1A78012A04
:10E8D00016D15B78012B13D100F000F988B1002527
:10E8E000ECB2A74205D821463046BDE8F840FFF714
:10E8F000CEBF301900F0D6F801350028F0D0F2E78D
:10E900000C20F8BD80C8FF1F08B540210248FFF762
:10E91000D7FF00F095F808BD83C8FF1F38B505463E
:10E9200000F0A8F80B28044609D140210548FFF75C
:10E93000C7FF28B92846BDE8384000F09BB800243E
:10E94000204638BDC3C8FF1F70B50C46461E0025C3
:10E950000CB9284670BD16F8010FFFF7DFFF013C28
:10E96000002818BF0B25A4B2F2E738B5451E0024D5
:10E9700015F8010F08B9204638BDFFF7CFFF002872
:10E9800018BF0B24F4E707B50123002200930649C2
:10E99000064B104600F020FA002814BF1B20002070
:10E9A00003B05DF804FB00BF05E80000E1E70000EC
:10E9B00038B50C46054600F097F8A0420AD32C441F
:10E9C0000020A54207D000B138BD15F8010B00F0BA
:10E9D00051F8F6E70B2038BD10B50A4A11784029E6
:10E9E0000ED05378D4180133DBB2402BA07001F164
:10E9F00001014FF00000117014BF5370507010BD32
:10EA00000B2010BD03C9FF1F10B50C4A117891B13E
:10EA100092F84230D4180133DBB2A4780470402B52
:10EA20004FF0000001F1FF31117014BF82F8423045
:10EA300082F8420010BD0A2010BD00BF03C9FF1FAD
:10EA4000014B1878704700BF03C9FF1F024B1878AD
:10EA5000C0F14000C0B2704703C9FF1F034B002242
:10EA60005A7083F842201A70704700BF03C9FF1F15
:10EA7000FFF7F4BF10B50A4A117840290ED0537839
:10EA8000D4180133DBB2402BA07001F101014FF02B
:10EA90000000117014BF5370507010BD0B2010BDDA
:10EAA00046C9FF1F10B50C4A117891B192F8423057
:10EAB000D4180133DBB2A4780470402B4FF000006F
:10EAC00001F1FF31117014BF82F8423082F8420028
:10EAD00010BD0A2010BD00BF46C9FF1F014B1878AA
:10EAE000704700BF46C9FF1F024B1878C0F14000B5
:10EAF000C0B2704746C9FF1F034B00225A7083F80B
:10EB000042201A70704700BF46C9FF1FFFF7F4BFCD
:10EB100070B50546007801F093F902780023D9B268
:10EB2000914207D25C1C03EB830303445E786B784D
:10EB30009E4227D1174C2B7A342202FB0142D67811
:10EB400013B334234B43E218907886420CD000F084
:10EB5000030204330C2010FB02302118205C0B89C7
:10EB60004A68497800F090FBD4F89C3083B12A467B
:10EB7000287812F8081F00290CBF03210521BDE8E1
:10EB8000704018472346CAE7937801339370D8E75B
:10EB900070BD00BF8CC9FF1F2DE9F04F85B00D4639
:10EBA00090468DF80F0001F04BF9022D064647D133
:10EBB000077800235C1CDBB2BB4210DB4FF000097E
:10EBC000DFF8B0B0CA465FFA89F4A74212DC284BDE
:10EBD000D3F89C30002B45D105B0BDE8F08F03EB96
:10EBE000830333440DF10F00DA78597801F0E2F92C
:10EBF0002346DFE704EB84043444E378A288617899
:10EC0000CDF804A0A07800900DF10F0001F0B0F94C
:10EC1000A378032B05D15A4661789DF80F0001F0C7
:10EC200031FA6178E37841F0100141EAC311002222
:10EC3000C9B20DF10F0001F0EDF909F10109C2E7C8
:10EC4000002DC4D10A490378342000FB03138A1C29
:10EC50003633294634329A42B9D002F8341C02F8CD
:10EC6000331CF7E7424629469DF80F009847B3E763
:10EC70008CC9FF1F11EB0000F0B40C7804F06004A5
:10EC8000202C1D4632D14C78042C1DD00AD8012CE2
:10EC900004D003D3022C20D0032C12D000202880D3
:10ECA000F0BC7047212C1BD004D8202CF6D1F0BC2E
:10ECB00000F040B9222C16D0232CEFD1F0BC00F08C
:10ECC00049B9F0BC00F049B902241C801468002541
:10ECD00025701468671C17606570F0BC00F056B9A9
:10ECE000F0BC00F01FB9F0BC00F076B9402C06D1A2
:10ECF000044CD4F8A04014B1A446F0BC6047CD2029
:10ED0000CEE700BF8CC9FF1F73B50446007801F041
:10ED100097F863680093A27A637A43EA0223ADF816
:10ED2000043002780023D9B2914207D25D1C03EB74
:10ED3000830303445E7863789E4225D1174D237A7E
:10ED4000342202FB0152D67803B334234B43EA1832
:10ED5000907886420CD000F0030204330C2010FBA4
:10ED600002302918285C0B894A68497800F08CFA2F
:10ED7000D5F89C3033B1227A20785AB104F10802D8
:10ED80000521984702B070BD2B46CCE7937801333C
:10ED90009370DAE76A460321F3E700BF8CC9FF1FCF
:10EDA00007B543680093437A817A43EA0123ADF8BB
:10EDB0000430084BD3F89C3002462BB1017A00781E
:10EDC00029B108320521984703B05DF804FB6A4673
:10EDD0000421F8E78CC9FF1F2DE9F84305460F46CB
:10EDE0001646984601F02CF802789DF82030013242
:10EDF0008146D2B20021284601F09EF80446E8B9C7
:10EE0000164A1749284600F086F999F80000154B74
:10EE1000342200FB022209F101011A4499463433DD
:10EE2000934201F105010CD14146284600F074F8E7
:10EE3000044618B9C9F89C70C9F8A0602046BDE81E
:10EE4000F88311F8050C03F8340C11F8040C03F8DE
:10EE5000330C03F8324C03F8314CE0E779EC000056
:10EE600099EB00008CC9FF1F08B5074B0022C3F8BF
:10EE70009C20C3F8A02000F0A1F918B9BDE8084013
:10EE800001F06EB808BD00BF8CC9FF1F2DE9F0412D
:10EE9000984605460E46174600F0D2FF0478002338
:10EEA000D9B2A14207D2013303EB8302024412F824
:10EEB000042CB242F4D1174C34234B43E218D078DF
:10EEC00092F802E0A0EB0E01C9B2042902D1C120E0
:10EED000BDE8F08100F003010130C0B24FF00C0C2E
:10EEE0000CFB0133D070A0EB0E001C44C0B2012813
:10EEF00025716671A760A4F80C8007D143463A4695
:10EF000031462846BDE8F04100F0BEB90020BDE81A
:10EF1000F08100BF8CC9FF1F014B002019607047B2
:10EF200030CAFF1F024B0979197100F08DBF00BF75
:10EF300030CAFF1F13B5002402AA1C80044B42F8FC
:10EF4000041D0979197100F08DFF02B010BD00BFDA
:10EF500030CAFF1F00201880704730B40C460221D1
:10EF6000198021796488084D012C297102D130BCA7
:10EF700000F08EBF022C02D130BC00F095BF002003
:10EF8000188030BC704700BF30CAFF1F30B40C4639
:10EF90000221198021796488074D012C297102D141
:10EFA00030BC00F08DBF022C02D130BC00F09ABF03
:10EFB0000020188030BC704730CAFF1F044B054A40
:10EFC00019795B791171137203210A23FFF75EBF70
:10EFD00030CAFF1F4EC0FF1FF8B500271F808B7877
:10EFE0000B4CA371C3F340035A0063F300020646BF
:10EFF0006271FFF7E3FF256845B1A37913F00202C0
:10F000001ABF3A46222121213046A8470020F8BDE8
:10F0100030CAFF1F034B00F108021B68007805216E
:10F02000184700BF38CAFF1F70B5094D04462A1D96
:10F03000012100F0D7FF80220121204600F0EAFFE5
:10F040002B68207800220A21BDE87040184700BFD5
:10F0500038CAFF1F37B501210DF10702044600F041
:10F06000C1FF9DF80730074D802B04D12A7901217B
:10F07000204600F0CFFF2B68207800220B21984714
:10F0800003B030BD38CAFF1F436805215A7800F02D
:10F09000C1BF73B50122002405460126002100F0FE
:10F0A00089FF334621468DE850001022284600F0A3
:10F0B0005FFF22462146284600F07CFF234621467A
:10F0C0008DE850001022284600F052FF31460222FF
:10F0D000284600F09FFF32460621284600F09AFF9E
:10F0E00022469021284600F095FF044B28781B68A3
:10F0F0002246214602B0BDE87040184738CAFF1FBB
:10F1000042783AB9C178C90141F0100101F090018B
:10F1100000F080BF704773B50C468DF8070001F012
:10F120000DFA1F4D2C600446002836D11D4A9DF86B
:10F130000700102100F0A6FF1B4A044612219DF88B
:10F14000070000F09FFF194A044314219DF80700AF
:10F1500000F098FFE4B20443154A9DF8070013211C
:10F1600000F090FFE4B20443124A9DF80700172113
:10F1700000F088FF02AEE4B204430F4A16F8010D16
:10F18000162100F07FFFE4B2044303220121304640
:10F1900000F040FF0323E4B22B71204602B070BDA3
:10F1A00038CAFF1F93F0000089F0000029F000002A
:10F1B00055F0000001F1000015F0000037B502AD78
:10F1C000174B05F8010D0022102128461A6000F0A7
:10F1D0005BFF12210446284600F056FF1421044329
:10F1E000284600F051FFE4B204431321284600F002
:10F1F0004BFFE4B204431721284600F045FFE4B278
:10F2000004431621284600F03FFFE4B2204310F0EB
:10F21000FF0003D19DF8070001F09CF903B030BD59
:10F2200038CAFF1F1FB501218DF807000DF10E022E
:10F230000DF1070000F0D6FE0DF10F0206210DF1D1
:10F24000070000F0CFFE9DF80E30802B18D19DF8FE
:10F250000F309B0714D59DF8070000F0EFFD012843
:10F2600004460DD172B60DF1070000F029FB002213
:10F2700021460DF107008DF80E2000F0CBFE62B69E
:10F280009DF80E0004B010BD73B50C4615461E4621
:10F290008DF80700FFF7C6FF802808D033462A46BE
:10F2A00021460DF1070000F0A7FA02B070BD002062
:10F2B000FBE77047062812D880000129C0B201D1AF
:10F2C0000230C0B2074AC0F34703122101FB0323F7
:10F2D0001A884FF6FF739A4208BFFF207047FF203D
:10F2E000704700BF40CAFF1F2DE9F041314C324D3D
:10F2F000324E4FF0000884F800814FF4107285F808
:10F3000040020F462846FF2101F0D6FF4FF48062ED
:10F3100041463046C5F8446201F0CEFF94F80C3106
:10F3200043F0800384F80C3194F80C311B06FBD4B5
:10F33000234BFF221A7094F80C3143F0400384F8F9
:10F340000C31204B196897B341F000411960194BFB
:10F35000310AC6F3074201F0FE0183F89C1083F8DE
:10F36000B020320E83F8B420174AC5F84822102284
:10F3700083F80821012283F89420BF2283F880209B
:10F3800093F8002102F07F0283F8002193F8842093
:10F3900042F0010283F8842093F8842042F01002A6
:10F3A00083F8842084221A770020BDE8F08121F0C0
:10F3B0000041CBE70020074040CAFF1F00D4FF1FD9
:10F3C00058C0FF1F0070044000D6FF1F0D4B93F87C
:10F3D0000C2102F0BF0283F80C21BF2283F88020A9
:10F3E00093F8842002F0FE0283F8842093F894209E
:10F3F00002F0FE0283F894201A7F02F07B021A7753
:10F400000020704700200740F7B5082304248DE84A
:10F410001800B1F803300D788878B3F5007F81BF0C
:10F420000023CB7002230B71062D71D8AB00DCB228
:10F43000012804BF0234E4B24FEA540E354C1227BF
:10F4400007FB0E474FF6FF76B7F800C0B4455FD113
:10F450004E78032E5CD801285AD897F80FC0BCF11B
:10F46000FF0F04BF4FF0000C87F80FC0B1F803C0C6
:10F47000122101FB0EFE04EB0E0743EA4003BA73B0
:10F48000FA7B7E7402F0010213435BB2D4F8482287
:10F49000C7F80220D9B2F9733874D4F8447224F84A
:10F4A0000EC01BB207EBC30E81F00101CEF80420A1
:10F4B000AEF802C04FF0080E07F833E007EBC10EBC
:10F4C000CEF80420AEF802C012FA8CF24FF0480ECB
:10F4D00007F831E0C4F8482228B917F8332062F061
:10F4E0007F0207F8332002AA02EB80002DB20A49FE
:10F4F00050F8082C11F82530012E0CBF164642F0AA
:10F5000001063343DBB201F82530002003B0F0BD23
:10F510009520FBE740CAFF1FC0200740084610B5F2
:10F520001146FFF7C7FEFF281DD0104B1221C0F374
:10F53000470001FB0030D3F84422C37B1CB283F0A8
:10F54000010312F8341001F07F0102F8341012F8B0
:10F55000331001F07F0102F833104FF0FF33837254
:10F56000C372002010BDC42010BD00BF40CAFF1FE1
:10F5700073B50C468DF80700114620461646FFF776
:10F5800099FEFF28054620D0214632460DF107009E
:10F59000FFF7C4FFC5F3470312210D4D59436B1804
:10F5A000D5F848221888121AC5F8482224B2094A08
:10F5B000002002F824004FF0FF326A549A705A700B
:10F5C000DA701A715A7102B070BD9620FBE700BF65
:10F5D00040CAFF1FC02007402DE9F0410E4680467B
:10F5E000114630461746FFF765FE0C4DC0F3470045
:10F5F000122303FB0050C47BFF2C0DD03A4631464A
:10F600004046FFF78BFF24B2D5F8442212F834307D
:10F6100063F07B0302F83430BDE8F08140CAFF1F7D
:10F6200010B5084600211446FFF744FE084AC0F30F
:10F630004700122101FB0020D2F84432C27B03EBC9
:10F64000C2035A68136823605368636010BD00BF2B
:10F6500040CAFF1F10B50C4620461146FFF72AFE90
:10F66000FF281AD024B2104B13F82430DBB213F069
:10F670000C0F12D09B0712D40C4BD3F8443213F862
:10F680003020D2090DD180F00100C0B213F8303023
:10F69000DB0914BF0320002010BD052010BD012090
:10F6A00010BD032010BD00BFC020074040CAFF1F8F
:10F6B00008B5FFF7FFFD074A1223C0F3470003FB1D
:10F6C0000020C37BFF2B1EBFD2F84422002102F88A
:10F6D000331008BD40CAFF1F2DE9F0410846002144
:10F6E00090461F46FFF7E6FD2249C0F3470012246B
:10F6F00004FB0014E57BFF2D39D022884FF6FF7004
:10F7000093B2834233D0D1F8441285F0010011F94D
:10F71000300000282BDB2EB287B901EBC603384638
:10F720005A80D4F802205A6011F8352002F04002C5
:10F7300062F0770201F83620BDE8F08101EBC602E5
:10F74000BB424FF0000028BF3B466781C4F80680EB
:10F75000207360735380C2F8048011F8353003F0D1
:10F76000400363F0770301F83630BDE8F081942060
:10F77000BDE8F08140CAFF1F2DE9F0410C46064666
:10F78000114620461546FFF795FD194BC0F347007B
:10F79000122202FB003090F80FE0BEF1FF0F24D0E0
:10F7A00027B2144A6CB1407C012D0CBF14211821E2
:10F7B000012818BF41F0010112F82700014302F8A7
:10F7C000271012F827106FF3410102F82710D3F821
:10F7D0004432002203F83E203DB92B462A462146FA
:10F7E0003046BDE8F041FFF777BFBDE8F08100BFCC
:10F7F00040CAFF1FC02007402DE9F0410C462046BB
:10F80000012117469846FFF755FDFF2836D01C4BBF
:10F81000C0F34700122202FB0030D3F8446290F894
:10F820000FE016F93E30002B28DB23B2154A12F800
:10F83000235015F0020521D10188C0F806701FFA87
:10F8400088F242818A42D8BF11460FFA8EF206EB47
:10F85000C2030573457359805F602CB9C82306F84D
:10F8600032302046BDE8F08116F83E3003F0400308
:10F8700063F0770306F832302C46F2E79324F0E782
:10F8800040CAFF1FC0200740034B044883F898106C
:10F890000122114600F0BEBB0020074080CCFF1FB4
:10F8A000054B0648002283F89420802283F80C211F
:10F8B0000121FF2200F0AEBB0020074080CCFF1FDB
:10F8C00038B51A4C94F8002102F07F0284F8002128
:10F8D00094F80C2102F0DF0284F80C2194F88020C7
:10F8E00042F0200284F8802094F8842002F0DF02A5
:10F8F00084F8842094F8942002F0DF0284F89420A5
:10F9000094F8942042F0040284F8942044F6206590
:10F91000013DADB200F0BCFE002DF9D194F8943059
:10F9200003F0FB0384F8943038BD00BF002007408B
:10F930002DE9F04FD84DD94C95F8807095F884306A
:10F9400095F8906087B0FF221F4094F840328DF800
:10F9500009208DF80C308DF80D20002301210DF1C8
:10F96000090204F510708DF80E3004938DF81530EF
:10F970008DF816308DF80F308DF8143000F032FB12
:10F9800095F80C31D907F6B20FD59DF80930802BC8
:10F990000BD195F8003103F07F0385F8003195F81D
:10F9A0000C3103F0DF0385F80C317A0711D5BA4B1F
:10F9B000042093F8A41093F8A02083F8800006ABED
:10F9C00042EA012223F80E2D03A91220049300F02D
:10F9D0006DFBFB074BD5B04DB0480123BF2685F822
:10F9E000803085F8886095F89430002743F0020352
:10F9F00085F894304FF4107285F89870FF2185F8DF
:10FA0000007101F059FC4FF480623946D4F8440289
:10FA100001F052FCD4F8443203F50073C4F84832C4
:10FA20009F4BFF221A7095F8943003F0FD0385F880
:10FA3000943095F80C3143F0400385F80C319F2346
:10FA400085F88C6085F8843095F8943003F0DF03F6
:10FA500085F8943003A9102000F028FB95F8943025
:10FA600003F0DF0385F8943007B0BDE8F08F3D0761
:10FA700040F19380884B082283F880203309C6F335
:10FA8000C000062B8DF80D308DF80F0000F2F480C9
:10FA9000C6F3800202EB830208B10232D2B2D4F87C
:10FAA000446206EBC201C2F34705D1F804E049887D
:10FAB000ADF81510122101FB0541CDF810E091F8C9
:10FAC0000FC08CF0010C81F80FC016F8321082F0D4
:10FAD000010A5FFA8AFAC1F380110FFA8AF881F0FD
:10FAE0000101890106EBC80906F83810002800F06A
:10FAF000D980DFF8ACB19BB99BF8002082B9FF2216
:10FB000019468BF8002003A81A460193FFF706FD5B
:10FB1000019B06F838301A46194603A8FFF7DCFDAA
:10FB20009BF80030012B04D09DF80D30002B00F025
:10FB3000AD80122101FB0541BDF815008B894A8972
:10FB400003449BB293428B8109D3B1F800E0C0B269
:10FB5000864540F09380897B012940F08F801221F7
:10FB600001FB0544D4F8061020881944D31A8342B7
:10FB7000D8BF98B2A9F80200C9F8041016F83A30B4
:10FB800003F0400363F0770306F83830424A92F8F6
:10FB9000943003F0DF0382F89430B80717D53E4C59
:10FBA000022384F8803094F8883094F88C2003A9DC
:10FBB000134016208DF8143000F078FABF2384F833
:10FBC000883094F8943003F0DF0384F89430F90619
:10FBD0001CD5314C202384F88030102384F88030E9
:10FBE00003A9142000F062FA94F80C3143F02003CA
:10FBF00084F80C3194F8003143F0800384F800312C
:10FC000094F8843043F0200384F88430BA060DD58C
:10FC1000214C202384F8803003A9132000F046FAF9
:10FC200094F8843003F0DF0384F884303B067FF5DA
:10FC30001BAF0DF10A02FF23102103A88DF80D3030
:10FC400000F0D0F99DF80A30134C012B04BF8DF859
:10FC50000F3000224FF0800308BF8DF80D2003A95C
:10FC600084F88030172000F021FA94F8943003F0E3
:10FC7000DF0384F89430F7E6FF2210E7122202FB3C
:10FC80000544D4F806200492ADF8153003A99DF878
:10FC90000D0000F00BFA79E70020074040CAFF1F73
:10FCA00058C0FF1F6BB916F832202F4902F03C02F2
:10FCB000342A35D101238DF80E309EF80030DB094F
:10FCC0000B70122101FB05414FF6FF734A899A42DE
:10FCD000DCD0BDF815E08B8973449BB28B81098819
:10FCE0008E4501D19A420CD88AB3B2FBF1F001FBE8
:10FCF000102080B258BB122000FB0540807B0128F9
:10FD000025D1D21A8A42D8BF91B2122202FB0544F1
:10FD1000C9B9D4F80230C9F80430A9F802102DE7A7
:10FD20000A78012ACDD1FF200870194603A8019353
:10FD3000FFF7F4FB019B06F838301A46194603A872
:10FD4000FFF7CAFCBDE7D4F806201344E3E712220C
:10FD500002FB0544D4F80620ADF815304FF0FF3310
:10FD60000492A372E37291E758C0FF1F13460A463C
:10FD7000194601F0A1BA00BF30B50329039C0498CD
:10FD80001DD12BB9164A226004220280002030BD0A
:10FD900040F209418B420FD1022A4FF000030CD8E8
:10FDA00010490C2505FB0313D9681B6951F8221073
:10FDB00021609B5C0380E9E701230122F0E707292A
:10FDC00001D9CD2030BD074B03EB8102126A2260BE
:10FDD000002AF6D003EB4103B3F84030EAE700BF56
:10FDE00059C0FF1F6815010001299FBF034B5B5CD1
:10FDF0001370002088BFCD20704700BF8CCCFF1F40
:10FE000001299DBF024B00205A54CD20704700BFEE
:10FE10008CCCFF1F19B14B1E58425841704701202E
:10FE20007047054B1A788A4204D05878431A5842D2
:10FE300058417047012070478CCCFF1F002070474D
:10FE400000487047B815010001299FBF044BC1EB62
:10FE5000C101C918002094BF1160CD20704700BFB8
:10FE60005DC0FF1F012930B50ED8084DC1EBC1019F
:10FE700008231068C45CC818284401330F2B00F80D
:10FE8000084CF6D1002030BDCD2030BD5DC0FF1F35
:10FE900001299FBF034B03EB41010020116088BF84
:10FEA000CD2070478ECCFF1F01299FBF034B03EB72
:10FEB00041010020116088BFCD20704792CCFF1F08
:10FEC00001290AD813681878054B03EB41018870A3
:10FED00013685B78CB7000207047CD20704700BF5F
:10FEE0008CCCFF1F01290AD813681878054B03EB47
:10FEF0004101887113685B78CB7100207047CD2079
:10FF0000704700BF8CCCFF1F084B5A7803F8022BB8
:10FF1000FF210022D1540132072AFBD1044A0023D9
:10FF2000052199540133072BFBD1704796CCFF1F55
:10FF30009FCCFF1F00BF7047013AD2B2062A10B50E
:10FF40001C4608D8054B5A70FFF7DEFF2146BDE876
:10FF50001040FFF7C9B9992010BD00BF96CCFF1F14
:10FF6000024B00225A70FFF731BA00BF96CCFF1F38
:10FF700037B50F4C257805B9C1B98DF802308DF829
:10FF800000109DF81830ADF8032069469DF81C203C
:10FF900000788DF80130FFF737FA9DF800301BB17B
:10FFA00010B92378013B237003B030BD9520FBE7E7
:10FFB00096CCFF1F38B50A4B0D461C7859788C42F9
:10FFC0001C4600D14DB929460078FFF7D1FA2DB172
:10FFD00020B923780133237038BD962038BD00BF87
:10FFE00096CCFF1F4B1E062B05D8094B19444B78A6
:10FFF000137000207047CB0607D501F00F010629CA
:020000021000EC
:1000000003D8034B19444B7AF2E78220704700BFB4
:1000100096CCFF1F4B1E062B2DE9F041804617465C
:1000200005D8174B19444A700020BDE8F081CB0673
:1000300022D501F00F05062D1ED8012A4FEAD11452
:100040000F4E06D122462946FFF7C6FA35446F7295
:10005000EAE7002AFAD173195B7A012BF6D122461E
:100060002946FFF789FB002DF0D184F001022946D3
:100070004046FFF781FBE9E78220BDE8F08100BF41
:1000800096CCFF1F00207047062903D9A1F1100369
:10009000072B07D8044B53F82130002B0CBFC4208A
:1000A00000207047C4207047E0150100102810B5EB
:1000B0000C4601D1FFF728FF034B53F820300BB15A
:1000C00020469847002010BDE01501001FB51446DA
:1000D00002228DF807001A8005210DF10F020DF1A3
:1000E0000700FFF77FFF034B9DF80F201A80236066
:1000F00004B010BDA8CCFF1F1FB5144601228DF817
:1001000007001A8004210DF10F020DF10700FFF71F
:1001100069FF044B9DF80F201A800020236004B073
:1001200010BD00BFA8CCFF1FF0B5002685B01E8013
:1001300049888DF80700ADF80E10FFF76BFE18B375
:10014000BDF80E20114F04ACB2FA82F2520901211F
:100150000DF10700FFF75EFF34F8022D0421D2B243
:100160000DF10700FFF756FF7B6822460121054687
:100170009DF8070098477B689DF8070032460221EA
:100180009847284605B0F0BD0425FAE7A8CCFF1F24
:1001900073B502AC002504F8010D0E461D80042243
:1001A00001212046FFF736FF7288024B28461A725B
:1001B00002B070BDA8CCFF1F13B54C8889888DE8AC
:1001C0000C000B46E2B2210AFFF7D6FD02B010BDCB
:1001D0002DE9F04186B017461E4606AA0023884640
:1001E000059303238DF80F0002F8083D01210DF15E
:1001F0000F00FFF7F7FE98F80050274C15F00305A5
:1002000028D10DF1110206210DF10F00FFF7EAFED2
:100210009DF811309DF80F0003F0030323800DF1CA
:100220001203019305AB00932A462B460221FFF7E8
:10023000A3FD059BDB7913F0400F238814BF43F027
:10024000010323F001032380022333803C6006B0C6
:10025000BDE8F081012D08D19DF81030012B02D1AD
:1002600098F80430ABB90023EDE7022DEED198F8F1
:10027000041041F010010DF11202C9B20DF10F008E
:10028000FFF7B0FE9DF8123003F0010323803580A4
:10029000DCE7CD20DAE700BFA8CCFF1F7FB5002246
:1002A0001A800B784E788DF8070013F003030D4683
:1002B000C6F3400634D1FEB14B88013B9BB2012B03
:1002C00052D80DF10F0206210DF10700FFF78AFE4B
:1002D000044670B9AB7801229A409DF80F301A435A
:1002E000D2B206210DF107008DF80F20FFF792FE24
:1002F0000446204604B070BD4E88012E34D10DF165
:100300000F0206210DF10700FFF76CFE04460028DE
:10031000EFD1AA7896409DF80F2022EA0602E0E786
:10032000022B21D109798DF80F10324641F01001CE
:100330000DF10700FFF76EFE6B78002E14BF07214A
:100340000821012B044607D19DF80F00C10900F0D8
:100350000F00FFF7ADF90821044B9DF807005B681B
:100360000DF10F029847C4E7CD24C2E7A8CCFF1FC8
:1003700010B500241C800B7803F00303012B05D17A
:100380008A780979FFF73CFD204610BD042010BD96
:1003900038B515460A7802F00302012A07D1054C48
:1003A0001A8009792246FFF71FFD2C6038BD042012
:1003B00038BD00BFA8CCFF1F13B5CD298DF80700AD
:1003C00007D1012290210DF10700FFF723FE02B0B3
:1003D00010BD0D491C88088A1268844288BF1880A5
:1003E0000C461B889DF807000021FEF74DFF94F98D
:1003F0000A30002BEBDA00231A4619460DF10700EC
:10040000FFF76AF9E3E700BFA8CCFF1F73B5054605
:1004100000266A4601218DF800600196FFF7E2FD93
:10042000AA78434C012A52D168680368C4F80A309C
:100430004368A07AC4F80E3004F10A0110F0600F8E
:100440001ED1E27A3B4B53F82240002C3DD09DF860
:100450000000022839D802EB42021344034493F807
:100460003430012B31D10DF1020301AA2878A047C5
:100470000DF1020301AA01462878FFF79DFF13E062
:10048000238AADF80230202B17D87BB102060DD499
:100490000A68C4F812204A68C4F81620314604F1EC
:1004A0001A022846FFF718F902B070BDE46B64B178
:1004B0000DF1020301AA2049D8E702A82B7800F821
:1004C000073D9021FFF7A6FDEEE7CD20D0E79DF890
:1004D0000030042B10D12B78217A02AD05F8063DAF
:1004E0002846FFF7D1F9012211462846FFF792FD71
:1004F000227A03212846E5E794F90A30002BD3DB62
:10050000EB78002BD0D1E66B86B1B5F809302878AE
:100510000833ADF8023004F112010DF1020301AA13
:10052000B04701460DF1020301AAA5E7CD21F9E785
:10053000A8CCFF1F40160100B2CCFF1F034B59602F
:10054000DA630021024AFFF79DBD00BFA8CCFF1F60
:100550000D04010007B502AB054A03F8010D0021A7
:1005600018465160D163FFF78FFD03B05DF804FBBF
:10057000A8CCFF1F00207047354B41F248015A5864
:1005800022F00D0242F005025A5041F204015A587D
:1005900042F480225A5041F234015A5842F48022E7
:1005A0005A5003F52C33602193F8942042F0020254
:1005B00083F89420C02283F80021FF221A7483F864
:1005C000802083F8882083F88420002283F88C2000
:1005D00083F80C111F491A75080A00F0FE0083F811
:1005E000982083F8C02083F8C42083F8C82083F8BB
:1005F000CC2083F8D02083F8D42083F8D82083F847
:10060000DC2083F8E02083F8E42083F8E82083F8F6
:10061000EC2083F8F02083F8F42083F8F82083F8A6
:10062000FC2083F89C00C1F30740090E83F8B0005A
:1006300083F8B41083F8AC201A7783F8082193F874
:10064000942002F0D40242F0010283F89420704713
:100650000070044000D4FF1F024B4FF400729A60F8
:10066000704700BF00E100E0034B4FF40072C3F895
:1006700088219A60704700BF00E100E008B5FEF7EE
:1006800082F910B9FFF7F0FF08BD1B2008BD00BFBD
:10069000034B4AF202629A814BF280429A81704780
:1006A00000200540844641EA000313F003036DD1A6
:1006B000403A41D351F8043B40F8043B51F8043B25
:1006C00040F8043B51F8043B40F8043B51F8043B2C
:1006D00040F8043B51F8043B40F8043B51F8043B1C
:1006E00040F8043B51F8043B40F8043B51F8043B0C
:1006F00040F8043B51F8043B40F8043B51F8043BFC
:1007000040F8043B51F8043B40F8043B51F8043BEB
:1007100040F8043B51F8043B40F8043B51F8043BDB
:1007200040F8043B51F8043B40F8043B51F8043BCB
:1007300040F8043B403ABDD2303211D351F8043B6B
:1007400040F8043B51F8043B40F8043B51F8043BAB
:1007500040F8043B51F8043B40F8043B103AEDD21A
:100760000C3205D351F8043B40F8043B043AF9D26B
:10077000043208D0D2071CBF11F8013B00F8013B3E
:1007800001D30B8803806046704700BF082A13D34B
:100790008B078DD010F003038AD0C3F10403D21A63
:1007A000DB071CBF11F8013B00F8013B80D331F897
:1007B000023B20F8023B7BE7043AD9D3013A11F817
:1007C000013B00F8013BF9D20B7803704B78437082
:1007D0008B7883706046704781F0004102E000BF73
:1007E00083F0004330B54FEA41044FEA430594EAF1
:1007F000050F08BF90EA020F1FBF54EA000C55EA2C
:10080000020C7FEA645C7FEA655C00F0E2804FEAFC
:100810005454D4EB5555B8BF6D420CDD2C4480EADE
:10082000020281EA030382EA000083EA010180EA0E
:10083000020281EA0303362D88BF30BD11F0004F5C
:100840004FEA01314FF4801C4CEA113102D0404292
:1008500061EB410113F0004F4FEA03334CEA1333CD
:1008600002D0524263EB430394EA050F00F0A780E5
:10087000A4F10104D5F1200E0DDB02FA0EFC22FAE0
:1008800005F2801841F1000103FA0EF2801843FAD4
:1008900005F359410EE0A5F120050EF1200E012AC5
:1008A00003FA0EFC28BF4CF0020C43FA05F3C01803
:1008B00051EBE37101F0004507D54FF0000EDCF17C
:1008C000000C7EEB00006EEB0101B1F5801F1BD325
:1008D000B1F5001F0CD349085FEA30004FEA3C0C29
:1008E00004F101044FEA445212F5800F80F09A801F
:1008F000BCF1004F08BF5FEA500C50F1000041EB23
:10090000045141EA050130BD5FEA4C0C404141EB26
:10091000010111F4801FA4F10104E9D191F0000F4D
:1009200004BF01460020B1FA81F308BF2033A3F1D0
:100930000B03B3F120020CDA0C3208DD02F1140CC7
:10094000C2F10C0201FA0CF021FA02F10CE002F102
:100950001402D8BFC2F1200C01FA02F120FA0CFCFB
:10096000DCBF41EA0C019040E41AA2BF01EB045144
:10097000294330BD6FEA04041F3C1CDA0C340EDC42
:1009800004F11404C4F1200220FA04F001FA02F385
:1009900040EA030021FA04F345EA030130BDC4F143
:1009A0000C04C4F1200220FA02F001FA04F340EA38
:1009B0000300294630BD21FA04F0294630BD94F0E9
:1009C000000F83F4801306BF81F480110134013DD0
:1009D0004EE77FEA645C18BF7FEA655C29D094EA41
:1009E000050F08BF90EA020F05D054EA000C04BFBF
:1009F0001946104630BD91EA030F1EBF00210020AA
:100A000030BD5FEA545C05D14000494128BF41F048
:100A1000004130BD14F580043CBF01F5801130BDAC
:100A200001F0004545F0FE4141F470014FF0000037
:100A300030BD7FEA645C1ABF194610467FEA655CE8
:100A40001CBF0B46024650EA013406BF52EA03358A
:100A500091EA030F41F4002130BD00BF90F0000F78
:100A600004BF0021704730B54FF4806404F13204B4
:100A70004FF000054FF0000150E700BF90F0000F6D
:100A800004BF0021704730B54FF4806404F1320494
:100A900010F0004548BF40424FF000013EE700BF64
:100AA00042004FEAE2014FEA31014FEA02701FBFF4
:100AB00012F07F4393F07F4F81F06051704792F0C6
:100AC000000F14BF93F07F4F704730B54FF4607440
:100AD00001F0004521F0004120E700BF50EA01028B
:100AE00008BF704730B54FF000050AE050EA010238
:100AF00008BF704730B511F0004502D5404261EBA8
:100B000041014FF4806404F132045FEA915C3FF4E8
:100B1000DCAE4FF003025FEADC0C18BF03325FEA81
:100B2000DC0C18BF033202EBDC02C2F1200300FA36
:100B300003FC20FA02F001FA03FE40EA0E0021FA5B
:100B400002F11444C1E600BF70B54FF0FF0C4CF445
:100B5000E06C1CEA11541DBF1CEA135594EA0C0FFB
:100B600095EA0C0F00F0DEF82C4481EA030621EA36
:100B70004C5123EA4C5350EA013518BF52EA033571
:100B800041F4801143F4801338D0A0FB02CE4FF023
:100B90000005E1FB02E506F00042E0FB03E54FF053
:100BA0000006E1FB03569CF0000F18BF4EF0010E4B
:100BB000A4F1FF04B6F5007F64F5407404D25FEA47
:100BC0004E0E6D4146EB060642EAC62141EA5551FA
:100BD0004FEAC52040EA5E504FEACE2EB4F1FD0C3C
:100BE00088BFBCF5E06F1ED8BEF1004F08BF5FEABA
:100BF000500E50F1000041EB045170BD06F000466C
:100C000046EA010140EA020081EA0301B4EB5C0418
:100C1000C2BFD4EB0C0541EA045170BD41F4801110
:100C20004FF0000E013C00F3AB8014F1360FDEBF35
:100C3000002001F0004170BDC4F10004203C35DA11
:100C40000C341BDC04F11404C4F1200500FA05F394
:100C500020FA04F001FA05F240EA020001F0004235
:100C600021F0004110EBD37021FA04F642EB0601AB
:100C70005EEA430E08BF20EAD37070BDC4F10C04D5
:100C8000C4F1200500FA04F320FA05F001FA04F299
:100C900040EA020001F0004110EBD37041F1000185
:100CA0005EEA430E08BF20EAD37070BDC4F1200590
:100CB00000FA05F24EEA020E20FA04F301FA05F2F8
:100CC00043EA020321FA04F001F0004121FA04F2A0
:100CD00020EA020000EBD3705EEA430E08BF20EA70
:100CE000D37070BD94F0000F0FD101F000464000AA
:100CF00041EB010111F4801F08BF013CF7D041EA2C
:100D0000060195F0000F18BF704703F0004652002F
:100D100043EB030313F4801F08BF013DF7D043EA00
:100D20000603704794EA0C0F0CEA135518BF95EAB6
:100D30000C0F0CD050EA410618BF52EA4306D1D13D
:100D400081EA030101F000414FF0000070BD50EA5C
:100D5000410606BF1046194652EA430619D094EAE6
:100D60000C0F02D150EA013613D195EA0C0F05D1D0
:100D700052EA03361CBF104619460AD181EA030124
:100D800001F0004141F0FE4141F470014FF00000DC
:100D900070BD41F0FE4141F4780170BD70B54FF077
:100DA000FF0C4CF4E06C1CEA11541DBF1CEA1355F7
:100DB00094EA0C0F95EA0C0F00F0A7F8A4EB0504D9
:100DC00081EA030E52EA03354FEA013100F08880D0
:100DD0004FEA03334FF0805545EA131343EA126399
:100DE0004FEA022245EA111545EA10654FEA00264E
:100DF0000EF000419D4208BF964244F1FD0404F507
:100E0000407402D25B084FEA3202B61A65EB030562
:100E10005B084FEA32024FF480104FF4002CB6EB1F
:100E2000020E75EB030E22BFB61A754640EA0C009F
:100E30005B084FEA3202B6EB020E75EB030E22BFDF
:100E4000B61A754640EA5C005B084FEA3202B6EB20
:100E5000020E75EB030E22BFB61A754640EA9C00DF
:100E60005B084FEA3202B6EB020E75EB030E22BFAF
:100E7000B61A754640EADC0055EA060E18D04FEA6D
:100E8000051545EA16754FEA06164FEAC30343EA0D
:100E900052734FEAC2025FEA1C1CC0D111F4801FDA
:100EA0000BD141EA00014FF000004FF0004CB6E7D3
:100EB00011F4801F04BF01430020B4F1FD0C88BF72
:100EC000BCF5E06F3FF6AFAEB5EB030C04BFB6EB7D
:100ED000020C5FEA500C50F1000041EB045170BD70
:100EE0000EF0004E4EEA113114EB5C04C2BFD4EB9D
:100EF0000C0541EA045170BD41F480114FF0000E21
:100F0000013C90E645EA060E8DE60CEA135594EA9C
:100F10000C0F08BF95EA0C0F3FF43BAF94EA0C0F9F
:100F20000AD150EA01347FF434AF95EA0C0F7FF414
:100F300025AF104619462CE795EA0C0F06D152EA68
:100F400003353FF4FDAE1046194622E750EA41064C
:100F500018BF52EA43067FF4C5AE50EA41047FF45D
:100F60000DAF52EA43057FF4EBAE12E74FEA4102C0
:100F700012F5001215D211D56FF47873B3EB6252EB
:100F800012D94FEAC12343F0004343EA505311F012
:100F9000004F23FA02F018BF404270474FF00000A4
:100FA000704750EA013005D111F0004008BF6FF0E2
:100FB000004070474FF00000704700BF80F00040D5
:100FC00002E000BF81F0004142001FBF5FEA410321
:100FD00092EA030F7FEA226C7FEA236C6AD04FEA21
:100FE0001262D2EB1363C1BFD21841404840414066
:100FF000B8BF5B42192B88BF704710F0004F40F418
:10100000000020F07F4018BF404211F0004F41F433
:10101000000121F07F4118BF494292EA030F3FD0FF
:10102000A2F1010241FA03FC10EB0C00C3F1200312
:1010300001FA03F100F0004302D5494260EB4000A1
:10104000B0F5000F13D3B0F1807F06D340084FEA0C
:10105000310102F10102FE2A51D2B1F1004F40EB01
:10106000C25008BF20F0010040EA03007047490069
:1010700040EB000010F4000FA2F10102EDD1B0FA34
:1010800080FCACF1080CB2EB0C0200FA0CF0AABF29
:1010900000EBC25052421843BCBFD04018437047C7
:1010A00092F0000F81F4000106BF80F400000132CD
:1010B000013BB5E74FEA41037FEA226C18BF7FEAA4
:1010C000236C21D092EA030F04D092F0000F08BFE6
:1010D0000846704790EA010F1CBF0020704712F0CD
:1010E0007F4F04D1400028BF40F00040704712F10C
:1010F00000723CBF00F50000704700F0004343F071
:10110000FE4040F4000070477FEA226216BF0846A6
:101110007FEA23630146420206BF5FEA412390EA69
:10112000010F40F4800070474FF0000304E000BF5F
:1011300010F0004348BF40425FEA000C08BF704710
:1011400043F0964301464FF000001CE050EA0102D4
:1011500008BF70474FF000030AE000BF50EA0102E9
:1011600008BF704711F0004302D5404261EB4101D6
:101170005FEA010C02BF84460146002043F0B643FB
:1011800008BFA3F18053A3F50003BCFA8CF2083A20
:10119000A3EBC25310DB01FA02FC634400FA02FC29
:1011A000C2F12002BCF1004F20FA02F243EB020030
:1011B00008BF20F00100704702F1200201FA02FC92
:1011C000C2F1200250EA4C0021FA02F243EB020085
:1011D00008BF20EADC707047FDF7A3FA002103E0A6
:1011E0000A4B5B584350043109480A4B42189A4253
:1011F000F6D3094A02E0002313600432074B9A42F7
:10120000F9D300F00DF8804770470000CC160100BC
:1012100008C0FF1F74C5FF1F00C6FF1F24D8FF1F93
:10122000224C08B5F7F72DF9F7F794F9F7F7EAFA32
:10123000F7F701FBF7F706FAF7F7B4FDFCF762FEE4
:10124000F8F733F8F7F798FBE08CF7F796FC20787F
:10125000F7F708FAE078F7F775FAF7F77FFD2189D5
:101260006079228AFCF7A2FEFDF782F9F8F7F6F919
:10127000FCF7DEFF0E4B04229A60F9F7A1FAFBF7A8
:10128000D1FF0C4B20229A60FBF728FCFCF79CF85E
:10129000FBF7C9FFF7F71EFDF7F750FD0028F3D065
:1012A000F8F7DCF9F9F78CFAEEE700BF0CC0FF1F86
:1012B000C0F00F4000F10F4070B4860746D0541EB6
:1012C000002A41D0CAB2034602E014F1FF343BD3F6
:1012D00003F8012B9D07F8D1032C2ED9CDB245EA96
:1012E00005250F2C45EA054519D903F110022646BC
:1012F000103E0F2E42F8105C42F80C5C42F8085C7D
:1013000042F8045C02F11002F2D8A4F1100222F0BB
:101310000F0204F00F041032032C13440DD91E46A3
:101320002246043A032A46F8045BFAD8221F22F028
:1013300003020432134404F003042CB1C9B21C4468
:1013400003F8011B9C42FBD170BC70471446034656
:10135000C2E700BF024B13B1024800F005B8704766
:101360000000000075130100002301461A461846CC
:1013700000F01EB838B50A4C0A4D641BA4100AD000
:1013800004F18043013B05EB8305013C55F804392A
:101390009847002CF9D1BDE8384000F08BB900BF68
:1013A000CC160100C8160100704700BF704700BF8F
:1013B0002DE9F8432C4D0646286898460F4691467D
:1013C000FFF7F2FF294B1C68D4F84831002B3ED0C0
:1013D0005A681F2A1CDC02F1010E76B103EB820170
:1013E0000124C1F88890D3F8880194402043022E4C
:1013F000C3F88801C1F8088123D00232C3F804E0A1
:10140000286843F82270FFF7D1FF0020BDE8F88379
:10141000174B0BB34FF4C870AFF300800346D8B13D
:10142000D4F848210260002141600A46C4F848010E
:101430004FF0010EC0F88811C0F88C11002EDCD0DE
:10144000CCE7D3F88C110C43C3F88C41D5E704F5F5
:10145000A673C4F84831BBE72868FFF7A7FF4FF031
:10146000FF30BDE8F88300BF70C5FF1FA416010060
:10147000000000008025000040380000004B000004
:10148000807000000096000000E10000002C0100C8
:1014900000C201000084030090D0030020A10700D7
:1014A00040420F0000000000E0930400C027090044
:1014B000FF00FF000000000064F00000E8030000EF
:1014C0001027000010270000140000000A00000090
:1014D00000000000FFFFFF3F00000100640000006B
:1014E0006400000000070000F4010000000000009C
:1014F00000000000000000000000000000000000EC
:10150000000000000050C3000088130001400808DC
:101510000000000000000000C80000000100000002
:101520000080000000000000000000000000C80073
:101530000020030000000000000000000000000088
:10154000C8000000000000000000000000000000D3
:10155000000000000000000000000000000000008B
:10156000000000000000000059C0FF1F0400000040
:1015700009040000CC150100DC150100000000008A
:1015800000000000000000000000000030C1FF1F4C
:10159000EDC0FF1F00000000000000000000000080
:1015A00000000000000000000000120043000000E6
:1015B0000000000000000000030102011000020210
:1015C00000100003030110000001000059C0FF1FBC
:1015D000B3C0FF1F8DC0FF1F6BC0FF1F043A262240
:1015E0000D04010009ED0000A1ED000011EB000069
:1015F00035FF000035FF000035FF000035FF00001B
:1016000035FF000035FF000035FF000035FF00000A
:1016100035FF000035FF000035FF000035FF0000FA
:1016200093F0000029F0000089F0000055F0000060
:1016300029F0000035FF000015F0000001F1000066
:10164000D10101009D020100000000009D02010087
:101650000000000091010100B9010100000000003C
:10166000F90001002901010091030100710301004B
:10167000CD00010001010001010000000001010096
:101680000000000001010101010000000101000152
:10169000010001000001000001000031313131562C
:1016A0003130380048C1FF1FF8B500BFF8BC08BC96
:1016B0009E467047F8B500BFF8BC08BC9E46704710
:0816C000551301003584000000
:0416C8001184000089
:1016CC009B16010000010200000800000100000050
:1016DC0002000000000000000000000000000000FC
:1016EC0000000000000000000000070000000000E7
:1016FC0000000000000000000000000000000000DE
:10170C00000000000101A120000000000200000008
:10171C00FF0403090400C2010000000800000000DF
:10172C0000000022034200410044002000530054FA
:10173C0000520049004E004700200049004E004472
:10174C0000450058002603530074006500700070BB
:10175C00006500720020004D006F0074006F007275
:10176C0000200044006500760020003A035400522B
:10177C000049004E0041004D004900430020004D3F
:10178C00006F00740069006F006E00200043006F52
:10179C00006E00740072006F006C002000200020AE
:1017AC00002000200009024300020100C03209049D
:1017BC0000000102020000052400100105240101B3
:1017CC00010424020605240600010705830310000A
:1017DC000A09040100020A0000000705810210003A
:1017EC0000070502021000001201000202000010A6
:1017FC003C2A000102000102000100000000000070
:10180C000000000034C4FF1F9CC4FF1F04C5FF1F51
:10181C0000000000000000000000000000000000BC
:10182C0000000000000000000000000000000000AC
:10183C00000000000000000000000000000000009C
:10184C00000000000000000000000000000000008C
:10185C00000000000000000000000000000000007C
:10186C00000000000000000000000000000000006C
:10187C00000000000000000000000000000000005C
:10188C00000000000000000000000000000000004C
:10189C00000000000000000000000000000000003C
:1018AC00000000000000000001000000000000002B
:1018BC000E33CDAB34126DE6ECDE05000B000000F0
:1018CC00000000000000000000000000000000000C
:1018DC0000000000000000000000000000000000FC
:1018EC0000000000000000000000000000000000EC
:1018FC0000000000000000000000000000000000DC
:0C1C2C00000000000000000000D8FF1FB6
:101C3800CC16010008C0FF1F6C0500000000000062
:081C4800000000000000000094
:020000020000FC
:020000041FFFDC
:04C00000000000003C
:04000003100011D9FF
:00000001FF
